:020000040001F9
:10900000C0590020159201001D9201001F9201001D
:10901000219201002392010025920100000000002E
:109020000000000000000000000000002792010086
:1090300029920100000000002B9201002D920100F6
:10904000719301002F920100159701002F920100EA
:109050002F920100000000002F9201002F920100CA
:109060002F9201002F920100E19601002F92010042
:109070002F9201002F9201002F9201002F920100E8
:109080002F920100C99301002F9201002F9201003D
:10909000ED9301002F920100F19301002F92010046
:1090A0002F9201002F92010000000000000000003C
:1090B0002F9201002F92010000000000000000002C
:1090C00000000000000000000000000000000000A0
:1090D0000000000000000000000000000000000090
:1090E0000000000000000000000000000000000080
:1090F0000000000000000000000000000000000070
:10910000000000000000000000000000000000005F
:10911000000000000000000000000000000000004F
:10912000000000000000000000000000000000003F
:10913000000000000000000000000000000000002F
:10914000000000000000000000000000000000001F
:10915000000000000000000000000000000000000F
:1091600000000000000000000000000000000000FF
:1091700000000000000000000000000000000000EF
:1091800000000000000000000000000000000000DF
:1091900000000000000000000000000000000000CF
:1091A00000000000000000000000000000000000BF
:1091B00000000000000000000000000000000000AF
:1091C000000000000000000000000000000000009F
:1091D000000000000000000000000000000000008F
:1091E000000000000000000000000000000000007F
:1091F000000000000000000000000000000000006F
:10920000DFF80CD000F04AF800480047351E020095
:10921000C05900200648804706480047FEE7FEE7A1
:10922000FEE7FEE7FEE7FEE7FEE7FEE7FEE7FEE716
:10923000F59301000192010040EA01039B0703D06E
:1092400009E008C9121F08C0042AFAD203E011F885
:10925000013B00F8013B521EF9D27047D2B201E047
:1092600000F8012B491EFBD270470022F6E710B52B
:1092700013460A4604461946FFF7F0FF204610BD84
:1092800030B504460020034600E05B1C934203D245
:10929000E05CCD5C401BF8D030BD0000064C074DB3
:1092A00006E0E06840F0010394E8070098471034B6
:1092B000AC42F6D3FFF7A8FF304202005042020052
:1092C00070B58C1810F8015B15F0070301D110F888
:1092D000013B2A1106D110F8012B03E010F8016BB5
:1092E00001F8016B5B1EF9D12B0705D40023521E38
:1092F0000DD401F8013BFAE710F8013BCB1A921CA0
:1093000003E013F8015B01F8015B521EF9D5A1429D
:10931000D8D3002070BD00F01F0201219140400908
:10932000800000F1E020C0F88012704700F01F02BA
:10933000012191404009800000F1E020C0F8801236
:10934000704700F01F02012191404009800000F1A8
:10935000E020C0F80011704700F01F020121914089
:109360004009800000F1E020C0F8001270470000C2
:1093700070B54FF48076304608F09EFD114CB5056F
:1093800060B1304608F09FFD0120C5F80803607900
:1093900020B9012060712168002088474FF482764F
:1093A000304608F089FD00280AD0304608F08BFDD1
:1093B0000220C5F808032168BDE870400120084775
:1093C00070BD00009C27002007480021C0F8401114
:1093D000C0F84411C0F84811C0F84C11C0F8001191
:1093E000C0F804110AF044BA001001400AF0B2B902
:1093F00008F0D0BFF0B5A848A74B012600781B1D88
:109400001A1D4FF0805106280BD11C78240708D173
:109410001478C4F30314032C06D0042C04D0052CB8
:1094200002D0062807D011E0B1F824439B4DC4F3C5
:1094300004242C6002E01C78240707D11478C4F3BC
:109440000314032C02D1974D954C6C67D1F8305121
:10945000D1F84442944FC4F342343C6006280CD106
:109460001C78240709D11478C4F30314032C04D105
:109470008E4C276827F0807727604FF080470024C4
:10948000C7F80C41C7F81041874F3F1F3C600628C2
:1094900007D11F783F0704D11778C7F30317032FAD
:1094A00002D0062808D01FE0DFF8FCC103270CF12A
:1094B000640CCCF8007007E01F783F0714D11778D0
:1094C000C7F30317032F0FD1DFF8E4C10527CCF84A
:1094D0000070774F78373E60754F08373C600CF16D
:1094E000040C3F27CCF80070724F3F68DFF8C8C10A
:1094F000CCF800706F4F3F1D3F680CF1040CCCF8A6
:1095000000706C4F08373F680CF1040CCCF8007009
:10951000684F0C373F680CF1040CCCF80070654FB5
:1095200010373F680CF1040CCCF80070614F143711
:109530003F680CF1040CCCF800705E4F18373F68A0
:10954000DFF874C10CF1200CCCF80070594F1C37B7
:109550003F680CF1040CCCF80070564F20373F6880
:109560000CF1040CCCF80070524F24373F680CF11A
:10957000040CCCF800704F4F28373F680CF1040CF6
:10958000CCF800704B4F2C373F680CF1040CCCF832
:109590000070484F30373F68DFF81CC10CF1400CB9
:1095A000CCF80070434F34373F680CF1040CCCF812
:1095B0000070404F38373F680CF1040CCCF8007055
:1095C0003C4F3C373F680CF1040CCCF80070394F2D
:1095D00040373F680CF1040CCCF80070DFF8DCC0B9
:1095E000FB27CCF80070062813D11F783F0710D155
:1095F0001778C7F30317032F03D0042F01D0052FCB
:1096000007D1D1F85872DFF8B8C007F04F07CCF88F
:1096100000702C480268D20702D06FF0010202608D
:10962000062D08D1D1F83401062804D12648016856
:1096300041F4806101604FF01021D1F80002002850
:1096400003DBD1F80402002822DA204A1660204801
:109650000368002BFCD01523C1F800320568002DEB
:10966000FCD0C1F8043201680029FCD01460016804
:109670000029FCD0BFF34F8F0C48F0380168154A21
:1096800001F4E06111430160BFF34F8F00BFFDE7BC
:10969000124911480860F0BDE00F00F0403501406C
:1096A0000DF0ADBA00C007403C050040FCED00E005
:1096B000105600400404001020C5004018F500407A
:1096C000E40E0040000400403C17004004E5014067
:1096D00000E401400400FA050090D003BC280020FB
:1096E0000A48D0F8441101290ED1D0F80413890397
:1096F0000AD50021C0F844110121C1600448427913
:109700000AB108F0EFB881717047000000A0004076
:1097100054280020014902480AF044BAEC330020E2
:109720000020004002E008C8121F08C1002AFAD138
:1097300070477047002001E001C1121F002AFBD1D1
:10974000704700000121202803DA814005480140CC
:1097500003E0402802DA2038814009B10120704737
:1097600000207047FC06FFBD082806D228B101285A
:1097700003D0042801D0012070470020704700006A
:109780001CB50E480D4C90F824002034C000207009
:1097900000206070A070204608F032FAE0700420CB
:1097A000ADF80400002200941146684609F0D4FD8B
:1097B000002802D0002000F027F81CBD542800200B
:1097C00038B5044600208DF80000684600F0FAF82D
:1097D0000A4884420CD0BFF34F8F09480168094AF8
:1097E00001F4E06111430160BFF34F8F00BFFDE75B
:1097F0009DF8000000F00AF938BD0000FECADDBA8D
:109800000CED00E00400FA050EB500210091CDE951
:1098100001106A4644F20100FFF7D2FF0EBD0000BE
:109820002DE9F84F2C4C8146924660880E468142C5
:109830004FD800274FF6FF788DF80070684600F08B
:10984000C1F822786078A188884201DA401C00E0E3
:109850000020C0B2904204D19DF8000000F0D6F87C
:1098600035E065786078884201DA401C00E000202D
:10987000607020786278824201D3101A02E0081AE0
:109880001044401CE18880B2884200D9E0809DF8F5
:10989000000000F0BBF8454519D0E068B9F1000FB1
:1098A00040F835A00DD066B161882069324605FBCD
:1098B00001004946FFF7C0FCE06800EBC500868068
:1098C00002E000EBC50087800020BDE8F88F04208F
:1098D000FBE70920F9E70000A427002010B50F4C92
:1098E00003E0401C00E000202070A068002814D194
:1098F00020786178814210D0227861882069E368FD
:1099000002FB010003EBC20153F832208988904723
:109910002078A1888842E6DAE3E710BDA42700207A
:1099200030B5CB0008339DB293074FF0000401D04F
:10993000072030BD054BDA602A441A615C701C7048
:1099400058809980DC80002030BD0000A4270020D2
:1099500008B500208DF80000684600F033F805498E
:109960008868421C01D0401C88609DF8000000F00F
:109970004DF808BDA4270020074801784078064A22
:109980008842928801D3401A02E0511A0844401CD0
:10999000101A80B270470000A427002008B50020EC
:1099A0008DF80000684600F00DF80548816809B19F
:1099B000491E81609DF8000000F028F808BD0000F5
:1099C000A427002030B5EFF3108172B60D4A9468D9
:1099D000012324B10370002900D162B630BD936029
:1099E0004FF0E023D3F88051074C25401560C3F8B1
:1099F0008041D3F8844154605A17C3F8842100226F
:109A00000270E8E71C350020FC06FFBD0B498A68A0
:109A1000002A11D000280FD1EFF3108072B60B6826
:109A20004FF0E022C2F800314B68C2F80431002246
:109A30008A60002800D162B6704700001C35002003
:109A40002DE9F041064608680C46411C4FF0A0473E
:109A50004FF0010506D005FA00F1C7F80815206897
:109A600008F029FB6068411C02D0002108F01AFBB5
:109A70003168A069C1F82405607D217D3268084302
:109A8000C2F86C05D4E900123068C0F80C15C0F8B3
:109A90001425207D012815D1A068411C02D0002189
:109AA00008F000FBE068411C05D08540C7F8085568
:109AB000E06808F000FBD4E902123068C0F808251D
:109AC000C0F81015BDE8F0812DE9FC471D460700E0
:109AD00090460E460AD036B10024019438780DF134
:109AE0000409692804D00720BDE8FC870E20FBE7A5
:109AF0000120134601904A4638460AF002F9002830
:109B0000F2D12B464A4631463846009405F0F6FF1E
:109B10000028E9D12B68C3B30025D8F800002C46F3
:109B2000232819D008DC012818D020280DD021289E
:109B30000DD0222816D10DE0402811D0412829D07F
:109B4000A02829D0A1280DD128E0164D00E0164DFF
:109B50009C1C07E0154DFBE7154DF9E7154D00E09E
:109B6000154D1C462038032806D84A46314638464B
:109B70000AF0FFF80028B7D123464A463146384656
:109B8000009507F001FD0028AED10198B04207D042
:109B90000920A9E7094DE4E7094DE2E7094DE0E7AF
:109BA0000020A1E7CBA70100FDCD010069E2010083
:109BB0002BCB0100D59B010099A7010015A701003F
:109BC000D3DF0100C5DF010013460A4601466920C4
:109BD00009F0A2B818B112B10BB10AF0CAB80E2040
:109BE000704738B568B162B15BB11C466B460AF08C
:109BF000C0F8002804D19DF8001001F00101217087
:109C000038BD0E2038BD08B551B14BB140B1007818
:109C100000F001008DF8000068460AF0B7F808BDB2
:109C20000E2008BD2DE9F84316465FEA00082BD048
:109C300056B34BB3164F1C460D46009707F0C2FCB7
:109C4000002822D1631C324629464046009707F07F
:109C5000B9FC002819D1A31C3246294640460AF017
:109C600088F8002811D1E31C3246294640460AF004
:109C700080F8002809D101B0231D3246294640460C
:109C8000BDE8F0430AF075B80E20BDE8F883000087
:109C9000B9F301002DE9F8431D4690460E002AD085
:109CA0004DB340B3154F0446009707F0DBFC002886
:109CB00022D12B4642463146601C009707F0D2FC69
:109CC000002819D12B4642463146A01C0AF05EF806
:109CD000002811D12B4642463146E01C0AF056F8C6
:109CE000002809D101B02B4642463146201DBDE86F
:109CF000F0430AF04BB80E20BDE8F883F7F30100FB
:109D00002DE9FC41164607000DD066B15BB11C463B
:109D10000D4601AB09F0F5FF002805D1019840B1CF
:109D2000216819B105E00E20BDE8FC8105F032FF85
:109D30002060201D0090234632462946384607F011
:109D4000B4FFF1E7F8B5144606000D461ED0ECB19D
:109D500000200090631C6A4630460AF00AF800288A
:109D600013D123466A46294630460AF002F80028F5
:109D70000BD1631D6A462946304609F0FAFF0028D8
:109D800003D10099A94200D00920F8BD0E20F8BDEA
:109D900017B581B0144669B164B1002000906B46DC
:109DA00001A8226809F0C4FF002801D100992160B0
:109DB00004B010BD0E20FBE728B111B10078602877
:109DC00003D0072070470E207047012901D00920D9
:109DD00070470020704713460A460146602008F08D
:109DE0009BBF30B49AB193B188B10488312C7ED036
:109DF00033DC182C76D01BDC132C4FD00FDC102C4E
:109E000067D007DC012C43D0022C71D13DE00E203D
:109E100030BC7047112C59D0122C69D13BE0142C66
:109E20003FD0152C43D0162C59D0172C60D141E0CF
:109E30001E2C51D008DC192C36D01A2C3DD01B2CEE
:109E400041D01C2C54D13BE0202C7DD0212C52D071
:109E5000222C4AD0302C4BD159E0323C262C47D210
:109E6000DFE804F04C4F6A525B6761586D5E70909A
:109E700090909090909090909090909090909090E2
:109E800090907E8184757B87788A30BC00F07EB8A4
:109E900030BC00F0C7B830BC01F0AEB830BC01F047
:109EA0002FBC30BC01F0BCBB30BC00F0F7BF30BCF5
:109EB00001F06EBA30BC00F0BDBF30BC01F0E2B8BA
:109EC00030BC01F027BB30BC01F0B2BC30BC01F0AB
:109ED0009BB930BC01F01CB930BC01F057BC30BCA0
:109EE00001F0DDB930BC01F00DBA30BC01E01DE07D
:109EF00048E001F091BA30BC01F0D4BA30BC03F0B4
:109F00005BB830BC03F096B930BC03F0C7B830BCC6
:109F100003F0C4BA30BC03F051BA30BC03F02EBB1E
:109F200030BC03F00FBC30BC03F0A2BC30BC03F06B
:109F300095BB30BC03F01EB930BC02F0B5BF30BCDD
:109F400003F0EAB930BC00E019E003F04CBC30BCCF
:109F500004F042BA30BC04F0BFBB30BC04F052BBCA
:109F600030BC04F0F9BB30BC04F0CCBA30BC04F017
:109F700073BB30BC04F0F0B930BC04F06CBA30BC38
:109F800001F004BB06200021196041E72DE9FE43E2
:109F90001D461646040007D036B12DB12088022890
:109FA00004D00720BDE8FE830E20FBE700270197C1
:109FB000D5F8008002200DF10409ADF808004B46E9
:109FC0004246314602A809F082FE0028EAD14B46FB
:109FD00042463146201D09F07AFE0028E2D14B4668
:109FE0004246314604F1080009F0D0FE0028D9D1DC
:109FF0004B464246314604F1100009F068FE002845
:10A00000D0D100974B4642463146E06805F0A4FDAA
:10A010000028C7D1A08805F05FFE0028C2D10199B1
:10A020002960BFE72DE9FC411D461646040007D014
:10A0300036B12DB12088012804D00720BDE8FC816D
:10A040000E20FBE7002000902F680120E846ADF8C5
:10A05000040043463A46314601A809F038FE00287C
:10A06000ECD143463A463146201D09F030FE002827
:10A07000E4D143463A46314604F1080009F086FE31
:10A080000028DBD100992960D8E77CB50C4640B1A7
:10A090002CB100230193057801A96D2D03D0072071
:10A0A0007CBD0E207CBD0125CDE9003513460A4656
:10A0B000214605F023FD0028F4D10198A04201D0EB
:10A0C00009207CBD00207CBD2DE9FF4182B098466F
:10A0D00014460F0028D03CB30020009025686D2066
:10A0E0006E468DF8040033462A4601A809F04EFE5C
:10A0F000002816D133462A46394602A809F018FE30
:10A1000000280ED1029848B95FEA080039462A466D
:10A11000334609D000F05AF8002802D10098206098
:10A12000002006B0BDE8F0810E20FAE71CB50C4611
:10A1300040B12CB100210191037801A96C2B03D00F
:10A1400007201CBD0E201CBD01230193074B00936B
:10A1500013460A46214605F0D1FC0028F3D10198A8
:10A16000A04201D009201CBD00201CBD7DA1010022
:10A1700013460A4601466C2008F0CEBD2DE9FC418D
:10A180001646070020D0FEB1F3B11C460D4601ABC8
:10A1900009F0EFFD002815D106200090631C32461F
:10A1A0002946384609F0FFFD00280BD19DF8042010
:10A1B000217862F3000121709DF80420520862F3B7
:10A1C00047012170BDE8FC810E20FBE72DE9FC4131
:10A1D0001D4617460E0013D095B188B1044600788D
:10A1E0008DF8040001A809F0D1FD002806D13B46F6
:10A1F00032460621601C009509F0EBFDBDE8FC81AC
:10A200000E20FBE72DE9F84316465FEA000813D05D
:10A2100096B18BB1094F1C460D46009707F0BEF969
:10A22000002807D104F1080332462946404600972A
:10A2300007F0B4F9BDE8F8830E20FBE7019D0100AB
:10A240002DE9FF41164607006ED0002E6CD0002B82
:10A250006AD0364800901C460D46384607F09EF9F5
:10A2600000285ED132480090231D324629463846E8
:10A2700005F044FC002854D104F108033246294675
:10A28000384609F03EFD00284BD104F10C0332465C
:10A290002946384609F00CFD002842D104F10E038E
:10A2A00032462946384609F064FD002839D104F1C8
:10A2B0000F00029005200090019002AB3246294623
:10A2C000384605F011FB00282BD104F11403324667
:10A2D0002946384609F04DFD002822D104F1150326
:10A2E00032462946384609F044FD002819D104F1C8
:10A2F000160332462946384609F03BFD002810D1A6
:10A3000003AB32462946384609F033FD002808D110
:10A310009DF80C20E17D62F30301120962F3041140
:10A32000E17504B0BDE8F0810E20FAE735A3010025
:10A330007DA10100F8B51646070019D0C6B1BBB122
:10A340001C460D4609F015FD002810D16B4632461B
:10A350002946384609F00DFD002808D19DF8002057
:10A36000617862F30001520862F341016170F8BD47
:10A370000E20F8BD2DE9FC411D46089C0E46070045
:10A3800037D036B10020019038780DF104087228DA
:10A3900002D00720BDE8FC81012001904AB310687B
:10A3A00038B335B3286820B31CB3206808B313480A
:10A3B000134600904246384605F0A0FB0028E9D13C
:10A3C0000F4800902B4642463146384605F096FB32
:10A3D0000028DFD10B4800902346424631463846DC
:10A3E00005F08CFB0028D5D10198B04203D009209C
:10A3F000D0E70E20CEE70020CCE70000733D02003E
:10A4000005A2010041A201002DE9FF4184B0984658
:10A4100014460F0019D0C4B10020019025687220A5
:10A4200001AE8DF8080033462A4602A809F0AEFCBA
:10A4300000280BD133462A46394604A809F078FC97
:10A44000002803D1049870B903E00E2008B0BDE8DD
:10A45000F0810748009033462A463946404605F0C9
:10A460007BFB0028F2D1019820600020EEE700007D
:10A470008D3D0200F8B51F460C46050008D02CB1F2
:10A480000020009028786E46732803D00720F8BD7E
:10A490000E20F8BD0120134600903246284609F0F0
:10A4A00068FC0028F5D13B4632462146284609F093
:10A4B00060FC0028EDD10098A04201D00920F8BD31
:10A4C0000020F8BD13460A460146732008F024BC5C
:10A4D00038B50C4640B12CB1002100910378694693
:10A4E000742B03D0072038BD0E2038BD0123009304
:10A4F00013460A46214609F03CFC0028F5D1009895
:10A50000A04201D0092038BD002038BD13460A46BC
:10A510000146742008F000BC7CB50C46D0B12CB1CB
:10A5200000230193057801A9792D01D007207CBD76
:10A530000125019572B1156865B1009313460A466D
:10A54000214605F0DBFA0028F1D10198A04203D0A2
:10A5500009207CBD0E207CBD00207CBD2DE9FF4183
:10A5600084B0984614460F0019D0C4B10020019061
:10A570002568792001AE8DF8080033462A4602A8E6
:10A5800009F004FC00280BD133462A46394604A8BA
:10A5900009F0CEFB002803D1049870B903E00E2027
:10A5A00008B0BDE8F0810748009033462A46394696
:10A5B000404605F0D1FA0028F2D101982060002031
:10A5C000EEE70000CF3C020038B50C46B8B12CB124
:10A5D0000021009103786946782B01D0072038BD0F
:10A5E000012300935AB113460A46214609F060FB45
:10A5F0000028F4D10098A04203D0092038BD0E20D5
:10A6000038BD002038BD13460A460146782008F0C0
:10A6100083BB2DE9FE431F46DDF828800C4605006C
:10A6200022D0F4B100200290287802AE802818D100
:10A6300001200290C2B1BFB113463246284609F04C
:10A6400037FB00280ED13B4632462146284609F00A
:10A6500090FB002806D1387840B1012808D00228A4
:10A6600008D00720BDE8FE830E20FBE7002202E0B1
:10A67000062200E010220092019243463246214613
:10A68000284605F031F90028ECD10298A04201D00B
:10A690000920E7E70020E5E713460A460146802047
:10A6A00008F03ABB2DE9FC411C460D46060025D0BA
:10A6B0002DB100200190307801AF7E2802D0072014
:10A6C000BDE8FC8101200190C2B1BCB12068A8B1F5
:10A6D00013463A46304609F0EBFA0028F0D1094813
:10A6E000009023463A462946304605F007FA0028EE
:10A6F000E6D10198A84203D00920E1E70E20DFE768
:10A700000020DDE795C7010013460A4601467E207A
:10A7100008F002BB2DE9FE4316465FEA000836D07A
:10A72000A6B39BB35F891B4800901C460D4640466C
:10A7300006F034FF002827D102AB324629464046B6
:10A7400009F017FB00281FD19DF8080004F1080349
:10A7500000F00300607032462946404609F0A8FA2E
:10A76000002811D104F10A0332462946404609F077
:10A770009FFA002808D12089231DCDE900703246B8
:10A780002946404605F0B0F8BDE8FE83FFE70E20FD
:10A79000FAE70000D1A901002DE9F04115460600B5
:10A7A00010D07DB173B11F460C465B1C09F0E1FA75
:10A7B000002808D13B462A4621463046BDE8F041F4
:10A7C00009F0D7BA0E20BDE8F0812DE9F041164618
:10A7D00007000FD076B16BB11C460D4609F0C9FADF
:10A7E000002808D1A31C324629463846BDE8F0416E
:10A7F00009F05EBA0E20BDE8F08100002DE9FC41B1
:10A800001C460D46060025D02DB100200190307861
:10A8100001AF752802D00720BDE8FC81012001901E
:10A82000C2B1BCB12068A8B113463A46304609F01F
:10A830003FFA0028F0D10948009023463A462946BD
:10A84000304605F05BF90028E6D10198A84203D014
:10A850000920E1E70E20DFE70020DDE76DA8010019
:10A8600013460A460146752008F056BA2DE9F04114
:10A87000164607001FD0F6B1EBB11C460D4609F095
:10A8800017FA002818D1A31C32462946384609F089
:10A890000FFA002810D1231D32462946384609F008
:10A8A00007FA002808D1A31D324629463846BDE8DC
:10A8B000F04109F0FDB90E20BDE8F0812DE9F0412D
:10A8C0001D4617460E001ED0EDB1E0B1044609F05A
:10A8D000FEF9002818D12B463A463146A01C09F053
:10A8E000F6F9002810D12B463A463146201D09F0D2
:10A8F000EEF9002808D12B463A463146A01DBDE8A6
:10A90000F04109F0E4B90E20BDE8F0812DE9FC41E9
:10A9100098460C46050021D02CB1002601962878D7
:10A9200001AF872802D00720BDE8FC8101200190FB
:10A93000A2B113463A46284609F0BAF90028F3D1E5
:10A9400043463A4621462846009605F0D7F80028A7
:10A95000EAD10198A04203D00920E5E70E20E3E701
:10A960000020E1E72DE9FF4184B01C461500884630
:10A970001AD0CCB1002001902668872001AF8DF855
:10A9800008003B463246294602A809F0FFF9002894
:10A990000BD13B463246294604A809F0C9F90028E4
:10A9A00003D1049870B903E00E2008B0BDE8F0812F
:10A9B000064800903B4632462946404605F0CCF812
:10A9C0000028F2D1019820600020EEE71DAA0100C6
:10A9D00038B5A0B19AB193B11C466B4609F0C9F9DC
:10A9E00000280BD19DF80020217862F3030121702B
:10A9F0009DF80020120962F30711217038BD0E2066
:10AA000038BD08B541B13BB130B100788DF80000D8
:10AA1000684609F0BBF908BD0E2008BDF8B51D4613
:10AA200017460E0012D08DB180B104460848009040
:10AA3000204606F0E5FD002809D101B02B463A4634
:10AA40003146601CBDE8F04009F0A0B90E20F8BD09
:10AA500003AA01002DE9FF5F1D460E9F144688469C
:10AA60005FEA000942D0B8F1000F07D0002602A823
:10AA7000CDE9010699F800006F2803D0072004B043
:10AA8000BDE8F09F012002907CB3206868B30068A5
:10AA900058B355B3286840B3006830B33B464146CD
:10AAA0004846019A09F065F90028E8D103AB414610
:10AAB0004846019A09F05DF90028E0D19DF80C00A4
:10AAC000012815D0266003AB41464846019A09F09B
:10AAD00050F90028D3D19DF80C0001281ED02E601B
:10AAE000029941452DD00920C9E7FFE70E20C6E7AE
:10AAF000D4F800A00024DFF850B00BE00AEB840388
:10AB0000CDF800B041464846019A04F0F7FF00280E
:10AB1000B5D1641C3878A042F0D8D4E72D68002461
:10AB20000A4E0AE005EB8403009641464846019A26
:10AB300004F0E4FF0028A2D1641C3878A042F1D8C8
:10AB4000CEE700209BE7000099B8010019B9010089
:10AB500013460A4601466F2008F0DEB82DE9FC4195
:10AB600090460C46050022D02CB10026019628788C
:10AB700001AF7D2802D00720BDE8FC8101200190B3
:10AB8000ABB10D4800903A46284604F0B7FF0028C4
:10AB9000F2D143463A4621462846009604F0AEFFDD
:10ABA0000028E9D10198A04203D00920E4E70E2053
:10ABB000E2E70020E0E70000B13C02002DE9FF439E
:10ABC00083B01E000E9C154689461BD0D4B10020D0
:10ABD0000190D4F800807D2001AF8DF808003B463D
:10ABE0004246314602A809F0D1F800280BD13B4675
:10ABF0004246314603A809F09BF8002803D1039888
:10AC0000C0B903E00E2007B0BDE8F0830B48009008
:10AC10003B4642463146284604F09EFF0028F2D1CA
:10AC200045B10097298843463246484609F0D1F895
:10AC30000028E8D1019820600020E4E7CF3C020022
:10AC40002DE9FC419846089E0C46050027D02CB102
:10AC500000200190287801AF7C2802D00720BDE8B1
:10AC6000FC8101200190D2B1B8F1000F17D0B6B12C
:10AC70000D48134600903A46284604F03FFF00284E
:10AC8000EDD143463A4621462846009607F00DF896
:10AC90000028E4D10198A04203D00920DFE70E206C
:10ACA000DDE70020DBE70000D1A9010013460A46DA
:10ACB00001467C2008F030B8F8B51F460C46050068
:10ACC00020D02CB10020009028786E46762801D044
:10ACD0000720F8BD01200090A2B19FB11346324673
:10ACE000284608F0E5FF0028F3D13B4632462146CE
:10ACF000284609F03EF80028EBD10098A04203D086
:10AD00000920F8BD0E20F8BD0020F8BD13460A4604
:10AD10000146762008F000B82DE9FC4116460700F0
:10AD200020D0FEB1F3B1102000901C460D463846ED
:10AD300009F039F8002813D101AB324629463846CC
:10AD400009F017F800280BD19DF80410227C4B085D
:10AD500061F3000263F34102890861F38702227400
:10AD6000BDE8FC810E20FBE72DE9FC411D4617469E
:10AD70000E001DD0E5B1D8B113460A460446102195
:10AD8000009509F026F8002810D1207C2B46C0F34E
:10AD90004002014662F35F0120F0030001438DF899
:10ADA00004103A46314601A808F0F0FFBDE8FC81E6
:10ADB0000E20FBE7F8B51646070014D09EB193B1FC
:10ADC0000A4800901C460D46384606F0E7FB00286E
:10ADD00008D10748009004F112033246294638464C
:10ADE00006F0DCFBF8BD0E20F8BD000019AD010037
:10ADF00075BC0100F8B51D4617460E0013D095B17D
:10AE000088B1044609480090204606F0F9FB002866
:10AE100008D1074800902B463A46314604F112000B
:10AE200006F0EEFBF8BD0E20F8BD000069AD010094
:10AE3000A3BC01002DE9FC411D461646040007D0C5
:10AE400036B12DB12088172804D00720BDE8FC8139
:10AE50000E20FBE7002000902F681720E846ADF891
:10AE6000040043463A46314601A808F030FF002866
:10AE7000ECD143463A463146201D08F028FF002811
:10AE8000E4D143463A46314604F1080008F07EFF1B
:10AE90000028DBD100992960D8E700002DE9FF41A7
:10AEA0001D461646040008D03EB135B12088192849
:10AEB00005D0072004B0BDE8F0810E20FAE700209D
:10AEC00001902F6819200DF10408ADF808004346E1
:10AED0003A46314602A808F0FAFE0028EAD1434675
:10AEE0003A463146201D08F0F2FE0028E2D116480D
:10AEF000009043463A46314604F1080006F076FBDE
:10AF00000028D7D1A08803A904F0A8FE18B100201A
:10AF100001992960CEE70D48009003980C49C0EBD9
:10AF2000001000EB800001EB800043463A463146BA
:10AF3000001D06F05BFB0028BCD1A08804F070FE69
:10AF40000028E5D0B6E7000055AF010019C60100A2
:10AF5000283500202DE9FC411D4690460E0045D0C5
:10AF6000F5B3E8B341780446C1F38002084662F3C2
:10AF70009F00C1F3C00140EAC1008DF804004246C1
:10AF80003146204608F002FF00282DD12B464246CC
:10AF9000314601A808F0FAFE002825D1144F2B46AF
:10AFA00042463146A01C009706F02AFB00281BD120
:10AFB0002B4642463146E01C009706F021FB002854
:10AFC00012D10C4F2B4642463146201D009706F009
:10AFD00017FB002808D12B4642463146601D00E091
:10AFE00004E0009706F00CFBBDE8FC810E20FBE7B7
:10AFF00055C60100CBC401002DE9FE431D4616468F
:10B00000040007D036B12DB12088122804D00720C3
:10B01000BDE8FE830E20FBE7002001902F68122080
:10B020000DF10408ADF8080043463A46314602A83F
:10B0300008F04DFE0028EBD143463A463146201D2C
:10B0400008F045FE0028E3D10648009043463A4602
:10B05000314604F1080006F0C9FA0028D8D1019958
:10B060002960D5E769B0010038B531B12BB120B105
:10B07000034C009406F0C4FA38BD0E2038BD000021
:10B08000BDA801002DE9FE431D461646040007D069
:10B0900036B12DB120881A2804D00720BDE8FE83E0
:10B0A0000E20FBE7002001902F681A200DF1040804
:10B0B000ADF8080043463A46314602A808F007FEBC
:10B0C0000028EBD143463A463146201D08F0FFFDEB
:10B0D0000028E3D10648009043463A46314604F141
:10B0E000080006F083FA0028D8D101992960D5E735
:10B0F000F5B0010038B531B12BB120B1034C00944B
:10B1000006F07EFA38BD0E2038BD00001DAA0100F1
:10B110002DE9FE431D461646040007D036B12DB179
:10B120002088102804D00720BDE8FE830E20FBE70E
:10B13000002001902F6810200DF10408ADF80800E0
:10B1400043463A46314602A808F0C1FD0028EBD13B
:10B1500043463A463146201D08F0B9FD0028E3D1A8
:10B160000648009043463A46314604F1080006F08E
:10B170003DFA0028D8D101992960D5E781B10100B5
:10B18000F8B51D4617460E0038D0BDB3B0B304461F
:10B190001B480090204606F033FA00282FD12B469A
:10B1A0003A463146E01D08F0F1FD002827D1154848
:10B1B00000902B463A46314604F1080006F020FA8A
:10B1C00000281CD12B463A46314604F1100008F005
:10B1D000DDFD002813D12B463A46314604F1180014
:10B1E00008F075FD00280AD101B02B463A463146D9
:10B1F00004F12000BDE8F04008F069BD0E20F8BD64
:10B20000CDA10100BDA801002DE9FF411D46164654
:10B21000040008D03EB135B12088112805D00720A0
:10B2200004B0BDE8F0810E20FAE7002001902F68FD
:10B2300011200DF10408ADF8080043463A463146A6
:10B2400002A808F044FD0028EAD143463A463146B8
:10B25000201D08F03CFD0028E2D10C480090434638
:10B260003A46314604F1080006F0C0F90028D7D16B
:10B27000A08803A904F0F2FC20B9A08804F0D0FC57
:10B280000028CDD1019900202960C9E791B20100C1
:10B2900019B113B108B108F079BD0E2070472DE93E
:10B2A000FC411D461646040007D036B12DB120885A
:10B2B000162804D00720BDE8FC810E20FBE7002003
:10B2C00000902F681620E846ADF8040043463A4641
:10B2D000314601A808F0FBFC0028ECD143463A4671
:10B2E0003146201D08F0F3FC0028E4D143463A46DD
:10B2F000314604F1080008F049FD0028DBD100992F
:10B300002960D8E72DE9FF411D461646040008D004
:10B310003EB135B12088182805D0072004B0BDE81B
:10B32000F0810E20FAE7002001902F6818200DF11F
:10B330000408ADF8080043463A46314602A808F032
:10B34000C6FC0028EAD1207B434600F001008DF8BE
:10B350000C003A463146201D08F0B9FC0028DDD12A
:10B360000A48009043463A463146A06804F0F4FB90
:10B370000028D3D143463A46314603A808F006FDDB
:10B380000028CBD101992960C8E700005BBC01000F
:10B390002DE9FF411D46904604000AD0B8F1000F88
:10B3A00007D035B12088152805D0072004B0BDE8A6
:10B3B000F0810E20FAE7002001902F68152001AEE1
:10B3C000ADF8080033463A46414602A808F07FFC33
:10B3D0000028EBD1A07B334600F001008DF80C0073
:10B3E0003A464146201D08F072FC0028DED13B465B
:10B3F0004246062104F10800009608F0EAFC002805
:10B40000D4D133463A46414603A808F0BFFC002891
:10B41000CCD101992960C9E72DE9FC411D461646AA
:10B42000040007D036B12DB12088222804D007208F
:10B43000BDE8FC810E20FBE7002000902F68222051
:10B44000E846ADF8040043463A46314601A808F004
:10B450003EFC0028ECD143463A463146201D08F018
:10B4600036FC0028E4D143463A46314604F1080050
:10B4700008F08CFC0028DBD143463A46314604F103
:10B48000090008F083FC0028D2D143463A463146F1
:10B4900004F10A0008F07AFC0028C9D1009929605B
:10B4A000C6E700002DE9FE431D461646040007D0FE
:10B4B00036B12DB12088212804D00720BDE8FE83B5
:10B4C0000E20FBE7002001902F6821200DF10408D9
:10B4D000ADF8080043463A46314602A808F0F7FBAB
:10B4E0000028EBD143463A463146201D08F0EFFBD9
:10B4F0000028E3D10648009043463A46314604F11D
:10B50000080006F073F80028D8D101992960D5E722
:10B5100019BF01002DE9FC411D461646040007D065
:10B5200036B12DB120881C2804D00720BDE8FC814D
:10B530000E20FBE7002000902F681C20E846ADF8A5
:10B54000040043463A46314601A808F0C0FB0028F3
:10B55000ECD143463A463146201D08F0B8FB00289E
:10B56000E4D143463A46314604F1080008F00EFCA7
:10B570000028DBD143463A46314604F1090008F081
:10B5800005FC0028D2D100992960CFE72DE9FE43C0
:10B590001D461646040007D036B12DB1208820285C
:10B5A00004D00720BDE8FE830E20FBE700200190B9
:10B5B0002F6820200DF10408ADF8080043463A46F4
:10B5C000314602A808F083FB0028EBD143463A46F7
:10B5D0003146201D08F07BFB0028E3D143463A4664
:10B5E000314604F1080008F0D1FB0028DAD10B48FD
:10B5F000009043463A46314604F10A0005F0F6FF52
:10B600000028CFD143463A46314604F1090008F0FC
:10B61000BDFB0028C6D101992960C3E7CDA1010077
:10B620002DE9FE431D461646040007D036B12DB164
:10B630002088142804D00720BDE8FE830E20FBE7F5
:10B64000002001902F6814200DF10408ADF80800C7
:10B6500043463A46314602A808F039FB0028EBD1B0
:10B6600043463A463146201D08F031FB0028E3D11D
:10B670000648009043463A46314604F1080005F07A
:10B68000B5FF0028D8D101992960D5E791B601000E
:10B690002DE9FC411D4617460E002AD04DB340B39C
:10B6A0000446807CC0F34002014662F35F01C0F3B0
:10B6B000800041EA80008DF804000F4800903A466F
:10B6C0003146204605F09CFF002810D10B48009021
:10B6D0002B463A46314604F1080005F091FF002858
:10B6E00005D12B463A46314601A808F04FFBBDE88C
:10B6F000FC810E20FBE70000CDA10100A3BC0100EE
:10B700002DE9FE431D461646040007D036B12DB183
:10B710002088132804D00720BDE8FE830E20FBE715
:10B72000002001902F6813200DF10408ADF80800E7
:10B7300043463A46314602A808F0C9FA0028EBD140
:10B7400043463A463146201D08F0C1FA0028E3D1AD
:10B750000648009043463A46314604F1080005F099
:10B7600045FF0028D8D101992960D5E771B70100BC
:10B7700038B531B12BB120B1034C009405F040FF36
:10B7800038BD0E2038BD000051C801002DE9FE4330
:10B790001D461646040007D036B12DB120881E285C
:10B7A00004D00720BDE8FE830E20FBE700200190B7
:10B7B0002F681E200DF10408ADF8080043463A46F4
:10B7C000314602A808F083FA0028EBD143463A46F6
:10B7D0003146201D08F07BFA0028E3D1064800908E
:10B7E00043463A46314604F1080005F0FFFE0028C2
:10B7F000D8D101992960D5E7FDB7010038B5A9B1C5
:10B80000A3B198B10078C0F34005044665F35F0426
:10B81000C0F3800544EA8504C0F3C00044EAC000D8
:10B820008DF80000684608F0B1FA38BD0E2038BD2A
:10B830002DE9FC411D461646040007D036B12DB156
:10B8400020881B2804D00720BDE8FC810E20FBE7E0
:10B85000002000902F681B20E846ADF80400434606
:10B860003A46314601A808F032FA0028ECD14346A6
:10B870003A463146201D08F02AFA0028E4D1434612
:10B880003A46314604F1080008F080FA0028DBD17E
:10B8900000992960D8E70000F8B51646070014D0D3
:10B8A0009EB193B10A4800901C460D46384605F0FB
:10B8B00075FE002808D10748009004F110033246B5
:10B8C0002946384605F06AFEF8BD0E20F8BD000096
:10B8D00019B901007DA10100F8B51D4617460E00FB
:10B8E00013D095B188B1044609480090204605F070
:10B8F00087FE002808D1074800902B463A4631467B
:10B9000004F1100005F07CFEF8BD0E20F8BD00002B
:10B910002FB90100CDA1010038B530B12AB123B152
:10B920001024009408F03FFA38BD0E2038BD08B549
:10B9300041B13BB130B1009313460A46102108F0E3
:10B9400048FA08BD0E2008BDF8B51F460C46050094
:10B9500020D02CB10020009028786E46822801D09B
:10B960000720F8BD01200090A2B19FB113463246D6
:10B97000284608F09DF90028F3D13B46324621467F
:10B98000284608F0F6F90028EBD10098A04203D031
:10B990000920F8BD0E20F8BD0020F8BD13460A4668
:10B9A0000146822007F0B8B92DE9FC411F460C463C
:10B9B000050023D02CB100200190287801AE812809
:10B9C00002D00720BDE8FC8101200190B2B1AFB1E7
:10B9D00013463246284608F06BF90028F2D1094890
:10B9E00000903B4632462146284604F087F800285E
:10B9F000E8D10198A04203D00920E3E70E20E1E757
:10BA00000020DFE715BA010013460A4601468120EF
:10BA100007F082B938B530B12AB123B1202400949F
:10BA200008F0C1F938BD0E2038BD00002DE9FC47F3
:10BA30009846DDF828900C46050031D02CB1002640
:10BA40000196287801AF832802D00720BDE8FC8743
:10BA50000120019022B35FEA090021D0B8F1000F64
:10BA60001ED013463A46284608F022F90028EDD1A8
:10BA70000D48009043463A462146284604F03EF8D9
:10BA80000028E3D14B463A4621462846009604F06A
:10BA900035F80028DAD10198A04203D00920D5E773
:10BAA0000E20D3E70020D1E745BC01002DE9FF417E
:10BAB00084B01C46150088461AD0CCB100200190F5
:10BAC0002668832001AF8DF808003B4632462946A0
:10BAD00002A808F05BF900280BD13B463246294604
:10BAE00004A808F025F9002803D1049870B903E0F0
:10BAF0000E2008B0BDE8F081064800903B46324673
:10BB00002946404604F028F80028F2D10198206028
:10BB10000020EEE7F9BB01002DE9FC479846DDF86F
:10BB200028900C46050031D02CB1002001902878D7
:10BB300001AE842802D00720BDE8FC8701200190D7
:10BB400022B3B8F1000F21D05FEA09001ED01346DE
:10BB50003246284608F0ACF80028EDD10D4F434698
:10BB6000324621462846009703F0C8FF0028E3D15B
:10BB70004B46324621462846009703F0BFFF002877
:10BB8000DAD10198A04203D00920D5E70E20D3E7EF
:10BB90000020D1E7A5BB010013460A4601468420D8
:10BBA00007F0BAB82DE9F84316465FEA00081ED040
:10BBB000EEB1E3B10F4800901C460D46404605F03B
:10BBC000EDFC002811D11027E31D324629464046DE
:10BBD000009708F0E8F8002807D104F1170332466F
:10BBE00029464046009708F0DEF8BDE8F8830E20AD
:10BBF000FBE700007DA10100F8B51D4617460E00C9
:10BC00001BD0D5B1C8B104460D480090204605F0C0
:10BC1000F7FC002810D13B4632461021E01D00956C
:10BC200008F0D7F8002807D13B463246102104F12E
:10BC30001700009508F0CDF8F8BD0E20F8BD000003
:10BC4000CDA1010038B530B12AB123B14024009410
:10BC500008F0A9F838BD0E2038BD08B541B13BB198
:10BC600030B1009313460A46402108F0B2F808BDEF
:10BC70000E2008BDF8B51646070010D07EB173B18E
:10BC80001C460D4608F014F8002807D10820009043
:10BC9000A31C32462946384608F085F8F8BD0E2028
:10BCA000F8BDF8B51D4617460E000ED06DB160B157
:10BCB000044608F00CF8002806D13B46324608211D
:10BCC000A01C009508F085F8F8BD0E20F8BD2DE900
:10BCD000F041164607000FD076B16BB11C460D46F9
:10BCE00007F0E6FF002808D1A31C32462946384653
:10BCF000BDE8F04107F0DCBF0E20BDE8F0812DE982
:10BD0000F0411D4617460E000ED06DB160B10446DD
:10BD100007F0DDFF002808D12B463A463146A01C2B
:10BD2000BDE8F04107F0D3BF0E20BDE8F081F8B5C3
:10BD30001646070010D07EB173B11C460D4607F0C1
:10BD4000B7FF002807D105200090A31C32462946E2
:10BD5000384608F028F8F8BD0E20F8BDF8B51D46A5
:10BD600017460E000ED06DB160B1044607F0AFFF6C
:10BD7000002806D13B4632460521A01C009508F05C
:10BD800028F8F8BD0E20F8BDF8B51646070018D003
:10BD9000BEB1B3B11C460D4607F08AFF00280FD193
:10BDA000A31C32462946384607F082FF002807D1F7
:10BDB00005480090231D32462946384603F09EFE72
:10BDC000F8BD0E20F8BD0000B13C0200F8B51D46DC
:10BDD00017460E0017D0B5B1A8B1044607F077FF9B
:10BDE00000280FD12B463A463146A01C07F06FFFC2
:10BDF000002807D1054800902B463A463146606836
:10BE000003F0AAFEF8BD0E20F8BD0000CF3C0200F2
:10BE10001CB538B132B12BB106240094019403F063
:10BE200063FD1CBD0E201CBD08B549B143B138B13E
:10BE3000009313460A460068062103F087FD08BDFB
:10BE40000E2008BDF8B51646070013D096B18BB189
:10BE50001C460D4607F02CFF00280AD16B463246DF
:10BE60002946384607F085FF002802D19DF80010CA
:10BE7000A170F8BD0E20F8BD2DE9FC411C460D4611
:10BE8000060025D02DB100200190307801AF8F2819
:10BE900002D00720BDE8FC8101200190C2B1BCB1F5
:10BEA0002068A8B113463A46304607F001FF002843
:10BEB000F0D10948009023463A462946304603F01F
:10BEC0001DFE0028E6D10198A84203D00920E1E731
:10BED0000E20DFE70020DDE7E9BE010013460A4639
:10BEE00001468F2006F018BF2DE9F04116460700E5
:10BEF0000FD076B16BB11C460D4607F03AFF002813
:10BF000008D1631C324629463846BDE8F04107F0A7
:10BF100030BF0E20BDE8F0812DE9F0411D461746E7
:10BF20000E000ED06DB160B1044607F02FFF00285F
:10BF300008D12B463A463146601CBDE8F04107F077
:10BF400025BF0E20BDE8F0817CB50C46E0B12CB1D8
:10BF500000230193057801A97B2D01D007207CBD2A
:10BF60000125019582B1156875B1022C0AD30093A1
:10BF700013460A46214603F0C1FD0028EFD101987F
:10BF8000A04203D009207CBD0E207CBD00207CBDDA
:10BF90002DE9FF4184B0984614460F0019D0C4B172
:10BFA0000020019025687B2001AE8DF80800334603
:10BFB0002A4602A807F0EAFE00280BD133462A469B
:10BFC000394604A807F0B4FE002803D1049870B9DC
:10BFD00003E00E2008B0BDE8F0810748009033462A
:10BFE0002A463946404603F0B7FD0028F2D10198B1
:10BFF00020600020EEE70000BDA801001CB50C4643
:10C00000C8B12CB100210191037801A97A2B01D08C
:10C0100007201CBD012301936AB1094B009313460D
:10C020000A46214603F06AFD0028F2D10198A04299
:10C0300003D009201CBD0E201CBD00201CBD00002B
:10C040006DA8010013460A4601467A2006F064BE38
:10C050001CB50C4640B12CB100210191037801A917
:10C06000712B03D007201CBD0E201CBD01230193A2
:10C07000074B009313460A46214603F03FFD002874
:10C08000F3D10198A04201D009201CBD00201CBDA5
:10C0900001C101002DE9FF4184B0984614460F000C
:10C0A00019D0C4B1002001902568712001AE8DF82F
:10C0B000080033462A4602A807F068FE00280BD184
:10C0C00033462A46394604A807F032FE002803D139
:10C0D000049870B903E00E2008B0BDE8F08107486D
:10C0E000009033462A463946404603F035FD002885
:10C0F000F2D1019820600020EEE7000055C1010058
:10C10000F8B51646070020D0FEB1F3B11C460D4627
:10C1100007F02FFE002817D1631C32462946384607
:10C1200007F027FE00280FD1A31C324629463846C7
:10C1300007F0BEFD002807D105480090231D3246B8
:10C140002946384603F0DAFCF8BD0E20F8BD0000A1
:10C1500019B90100F8B51D4617460E001FD0F5B1FC
:10C16000E8B1044607F012FE002817D12B463A46E4
:10C170003146601C07F00AFE00280FD12B463A46D4
:10C180003146A01C07F0A3FD002807D10548009008
:10C190002B463A463146606803F0DEFCF8BD0E20BF
:10C1A000F8BD00002FB901001CB50C4640B12CB100
:10C1B00000210191037801A9702B03D007201CBD39
:10C1C0000E201CBD01230193074B009313460A4622
:10C1D000214603F093FC0028F3D10198A04201D03E
:10C1E00009201CBD00201CBD01C1010013460A46E8
:10C1F0000146702006F090BD2DE9FC471D460A9CC3
:10C200000E46070035D046B14FF00008CDF8048047
:10C2100038780DF104098E2802D00720BDE8FC878C
:10C22000012001902AB325B3286810B313464A466B
:10C23000384607F03DFD0028F0D12B464A463146EE
:10C240003846CDF8008003F059FC0028E6D184B1CF
:10C25000206870B123464A4631463846CDF8008002
:10C2600003F04CFC0028D9D10198B04203D009203A
:10C27000D4E70E20D2E70020D0E700002DE9FF47E9
:10C2800084B09946DDF840A014465FEA01081AD050
:10C29000CCB10020019026688E2001AF8DF80800F7
:10C2A0003B463246414602A807F070FD00280BD1FC
:10C2B0003B463246414604A807F03AFD002803D128
:10C2C0000498B8B903E00E2008B0BDE8F0870B4D24
:10C2D0003B46324641464846009503F03DFC002867
:10C2E000F2D13B46324641465046009503F034FCBD
:10C2F0000028E9D1019820600020E5E78D3D02008B
:10C300002DE9F8431F46DDF820800C4605002CD0AF
:10C310002CB10020009028786E46882802D0072093
:10C32000BDE8F88301200090FAB1F7B15FEA080098
:10C330001BD013463246284607F0BAFC0028EFD13E
:10C340003B4632462146284607F013FD0028E7D138
:10C35000434632462146284607F00BFD0028DFD130
:10C360000098A04203D00920DAE70E20D8E7002089
:10C37000D6E713460A460146882006F0CDBC38B5FC
:10C380000C46B8B12CB10021009103786946892B85
:10C3900001D0072038BD012300935AB113460A4645
:10C3A000214607F085FC0028F4D10098A04203D074
:10C3B000092038BD0E2038BD002038BD13460A467E
:10C3C0000146892006F0A8BC2DE9FC471E46DDE9A0
:10C3D0000A540F465FEA000842D03FB100200190A6
:10C3E00098F800000DF10409862802D00720BDE866
:10C3F000FC870120019092B38EB385B37CB3306883
:10C4000068B3286858B3206848B313464A46404684
:10C4100007F04EFC0028EAD11348009033464A4604
:10C420003946404603F06AFB0028E0D10F480090EF
:10C430002B464A463946404603F060FB0028D6D1D9
:10C440000B48009023464A463946404603F056FBC7
:10C450000028CCD10198B84204D00920C7E7FFE7F3
:10C460000E20C4E70020C2E719AD010019B9010090
:10C47000F1C8010013460A460146862006F04CBC6E
:10C4800038B500B3FAB1F3B11C466B4607F071FC46
:10C49000002817D19DF80020217862F30001217057
:10C4A0009DF80020520862F3410121709DF80020A0
:10C4B000920862F3820121709DF80020D20862F395
:10C4C000C301217038BD0E2038BD38B5A9B1A3B164
:10C4D00098B10078C0F34005044665F35F04C0F3EB
:10C4E000800544EA8504C0F3C00044EAC0008DF82A
:10C4F0000000684607F04AFC38BD0E2038BD000039
:10C50000F8B51646070029D046B33BB3144800904F
:10C510001C460D46384603F0F1FA00281DD111489B
:10C520000090231D32462946384603F0E7FA0028DA
:10C5300013D10D48009004F10803324629463846CD
:10C5400003F0DCFA002808D10848009004F10C033D
:10C5500032462946384603F0D1FAF8BD0E20F8BD20
:10C56000B5AD010099B80100F1C8010045BC01005A
:10C57000F8B51D4617460E0026D02DB320B304464D
:10C5800012480090206803F0E7FA00281BD11048F9
:10C5900000902B463A463146606803F0DDFA0028E9
:10C5A00011D10C4800902B463A463146A06803F062
:10C5B000D3FA002807D1084800902B463A46314666
:10C5C000E06803F0C9FAF8BD0E20F8BDF5AD010032
:10C5D000D9B8010007C901005BBC01002DE9F8438F
:10C5E00016465FEA000813D096B18BB1094F1C467E
:10C5F0000D46009704F0D2FF002807D104F1100384
:10C60000324629464046009704F0C8FFBDE8F8834B
:10C610000E20FBE701C501002DE9F8431D469046B9
:10C620000E0012D08DB180B1094F0446009704F07E
:10C63000E7FF002807D12B464246314604F110009F
:10C64000009704F0DDFFBDE8F8830E20FBE7000053
:10C6500071C5010038B5A9B1A3B198B10078C0F394
:10C660004005044665F35F04C0F3800544EA850491
:10C67000C0F3C00044EAC0008DF80000684607F02F
:10C6800085FB38BD0E2038BD2DE9FC479846DDE915
:10C690000A540E4607003FD036B10020019038788A
:10C6A0000DF104097F2802D00720BDE8FC87012096
:10C6B000019082B3B8F1000F2ED065B3286850B353
:10C6C0004CB3206838B313464A46384607F0F0FAB0
:10C6D0000028EAD143464A463146384607F049FB2E
:10C6E0000028E2D10E4800902B464A463146384693
:10C6F00003F004FA0028D8D10A48009023464A469D
:10C700003146384603F0FAF90028CED10198B042FC
:10C7100004D00920C9E7FFE70E20C6E70020C4E7E0
:10C7200095C70100DDC501002DE9FF4184B09846A1
:10C7300014460F0019D0C4B10020019025687F2055
:10C7400001AE8DF8080033462A4602A807F01EFB0A
:10C7500000280BD133462A46394604A807F0E8FAE8
:10C76000002803D1049870B903E00E2008B0BDE89A
:10C77000F0810748009033462A463946404603F088
:10C78000EBF90028F2D1019820600020EEE70000CC
:10C7900019C601002DE9FC4116465FEA000853D096
:10C7A000002E51D0002B4FD01C460D4601AB07F098
:10C7B000E0FA002846D1631C32462946404607F07D
:10C7C000D8FA00283ED1A31C32462946404607F03D
:10C7D000D0FA002836D11D4FE31C32462946404688
:10C7E000009704F0DBFE00282CD1231D3246294699
:10C7F0004046009704F0D2FE002823D19DF8042083
:10C80000217862F3000121709DF80420520862F340
:10C81000410121709DF80420920862F38201217089
:10C820009DF80420D20862F3C30121709DF8042012
:10C83000120962F3061121709DF80420D20962F3F7
:10C84000C7112170BDE8FC810E20FBE781C4010007
:10C850002DE9FC411D4690460E0045D0F5B3E8B3E6
:10C8600004460078C0F34002014662F35F01C0F362
:10C87000800241EA8201C0F3C00241EAC201C0F372
:10C88000021241EA021120F07F0001438DF80410EA
:10C890004246314601A807F079FA002822D12B46FA
:10C8A00042463146601C07F071FA00281AD12B4627
:10C8B00042463146A01C07F069FA002812D10B4FFE
:10C8C0002B4642463146E01C009704F099FE0028B2
:10C8D00008D12B4642463146201D00E004E0009777
:10C8E00004F08EFEBDE8FC810E20FBE7CBC4010006
:10C8F00038B530B12AB123B11024009407F053FAAF
:10C9000038BD0E2038BD08B541B13BB130B1009300
:10C9100013460A46102107F05CFA08BD0E2008BD38
:10C920002DE9F8439846089F0C46050028D02CB105
:10C930000020009028786E46772802D00720BDE8B6
:10C94000F88301200090DFB113463246284607F0F5
:10C9500010FA0028F3D1434632462146284607F014
:10C96000A7F90028EBD13B4632462146284607F07E
:10C9700000FA0028E3D10098A04203D00920DEE7A6
:10C980000E20DCE70020DAE713460A46014677204E
:10C9900006F0C2B92DE9FE4F1446060098460D4632
:10C9A00029D035B10027019730780DF1040A6E289F
:10C9B00002D00720BDE8FE8F01200190DCB1206885
:10C9C000C8B10068B8B15246304607F0D2F9002825
:10C9D000F0D102AB52462946304607F0CAF900288A
:10C9E000E8D19DF80800012807D027600198A842E7
:10C9F00019D00920DEE70E20DCE727680024DFF8E5
:10CA00002C900BE007EB8403524629463046CDF8C4
:10CA1000009003F073F80028CCD1641C98F8000053
:10CA2000A042EFD8E2E70020C4E700007DA10100AA
:10CA300013460A4601466E2006F06EB938B5A0B11D
:10CA40009AB193B11C466B4607F093F900280BD1BD
:10CA50009DF80020217862F3000121709DF80020EC
:10CA6000520862F34101217038BD0E2038BD38B53F
:10CA700090B38AB383B31C466B4607F07AF900285B
:10CA800029D19DF80020217862F3000121709DF8E2
:10CA90000020520862F3410121709DF800209208A5
:10CAA00062F3820121709DF80020D20862F3C30175
:10CAB00021709DF80020120962F3041121709DF885
:10CAC0000020520962F3451121709DF8002092095F
:10CAD00062F38611217038BDFFE70E20FBE738B501
:10CAE00009B303B3F8B10078C0F34005044665F319
:10CAF0005F04C0F3800544EA8504C0F3C00544EA3E
:10CB0000C504C0F3001544EA0514C0F3401544EA17
:10CB10004514C0F3801044EA80108DF80000684688
:10CB200007F034F938BD0E2038BD18B112B10BB181
:10CB300007F0BEB80E207047F8B51D4617460E0028
:10CB40000FD075B168B1044607F0C1F8002807D1CD
:10CB5000054800902B463A463146A01C04F064FD7F
:10CB6000F8BD0E20F8BD0000D7F40100F8B51D4651
:10CB700017460E000FD075B168B1044607F0A7F84C
:10CB8000002807D1054800902B463A463146A01CA4
:10CB900004F04AFDF8BD0E20F8BD0000F1F60100DA
:10CBA0002DE9FC411C460D46060025D02DB1002084
:10CBB0000190307801AF9F2802D00720BDE8FC81AA
:10CBC00001200190C2B1BCB12068A8B113463A4619
:10CBD000304607F06DF80028F0D109480090234650
:10CBE0003A462946304602F089FF0028E6D10198EE
:10CBF000A84203D00920E1E70E20DFE70020DDE7AF
:10CC0000BFD9010013460A4601469F2006F084B8AA
:10CC10002DE9FC411D4617460E0032D085B378B38E
:10CC2000044619480090204604F0FEFC002825D157
:10CC3000164800902B463A463146201D04F0F4FC7D
:10CC400000281BD160792B4600F001008DF804000C
:10CC50003A46314601A807F099F800280ED12B4634
:10CC60003A463146A01D07F032F8002806D12B467F
:10CC70003A46314604F1080007F029F8BDE8FC8186
:10CC8000FFE70E20FAE70000F1F60100DFCA01001D
:10CC90002DE9FC411D46089C0E46070033D036B1F5
:10CCA0000020019038780DF10408A02802D0072058
:10CCB000BDE8FC81012001902AB325B3286810B398
:10CCC0000CB32068F8B113464246384606F0F0FF30
:10CCD0000028EDD10E4800902B464246314638469A
:10CCE00002F00CFF0028E3D10A4800902346424698
:10CCF0003146384602F002FF0028D9D10198B042EF
:10CD000003D00920D4E70E20D2E70020D0E70000AE
:10CD1000C1F60100BFD9010013460A460146A02012
:10CD200005F0FABF2DE9FC411C46089F0D460600A0
:10CD300026D035B10020019030780DF10408A228EA
:10CD400002D00720BDE8FC8101200190C2B1BCB136
:10CD50002068A8B1A7B113464246304606F0A8FFA6
:10CD60000028EFD12346424629463046009704F07A
:10CD7000CFF80028E6D10198A84203D00920E1E7C6
:10CD80000E20DFE70020DDE713460A460146A22019
:10CD900005F0C2BF2DE9FC411F460C46050009D035
:10CDA0002CB100200190287801AE9D2804D00720E6
:10CDB000BDE8FC810E20FBE70120134601903246BE
:10CDC000284606F075FF0028F2D1084800903B463F
:10CDD00032462146284602F091FE0028E8D101980B
:10CDE000A04201D00920E3E70020E1E7BFD901001C
:10CDF00013460A4601469D2005F08EBF18B112B1B8
:10CE00000BB106F0B6BF0E2070470000F8B51D4606
:10CE100017460E000FD075B168B1044606F057FFF3
:10CE2000002807D1054800902B463A463146A01C01
:10CE300004F0FAFBF8BD0E20F8BD0000F1F6010089
:10CE40002DE9FC411F460C46050009D02CB10020FD
:10CE50000190287801AE9E2804D00720BDE8FC810F
:10CE60000E20FBE70120134601903246284606F0CB
:10CE70001FFF0028F2D1084800903B463246214669
:10CE8000284602F03BFE0028E8D10198A04201D0DC
:10CE90000920E3E70020E1E7BFD9010013460A4675
:10CEA00001469E2005F038BF2DE9FE431D4616467B
:10CEB000040007D036B12DB12088342804D00720D3
:10CEC000BDE8FE830E20FBE7002001902F68342090
:10CED0000DF10408ADF8080043463A46314602A871
:10CEE00006F0F5FE0028EBD143463A463146201DB8
:10CEF00006F0EDFE0028E3D143463A463146A01D38
:10CF000006F0E5FE0028DBD143463A46314604F1FF
:10CF1000080006F0DCFE0028D2D107480090434606
:10CF20003A46314604F10A0004F074FB0028C7D1E8
:10CF300001992960C4E700003DCF01002DE9F843C5
:10CF40001F4691465FEA010814D09FB190B1044694
:10CF500006F0BDFE00280ED13B464A464146A01CC5
:10CF600006F014FF002806D1A178012905D0104E43
:10CF7000002515E00E20BDE8F8830E4EF8E7A078F6
:10CF8000012811D005EBC50004EB4000001D3B4615
:10CF90004A464146009604F047FB0028EBD16D1C41
:10CFA0002188A942EBD8E6E705EB4500ECE7000055
:10CFB00039CB01006DCB01002DE9FE431D4616461D
:10CFC000040007D036B12DB12088322804D00720C4
:10CFD000BDE8FE830E20FBE7002001902F68322081
:10CFE0000DF10408ADF8080043463A46314602A860
:10CFF00006F06DFE0028EBD143463A463146201D2F
:10D0000006F065FE0028E3D143463A463146A01DAE
:10D0100006F05DFE0028DBD143463A46314604F176
:10D02000080006F054FE0028D2D10748009043467D
:10D030003A46314604F10A0004F0ECFA0028C7D160
:10D0400001992960C4E700004DD001002DE9F843A3
:10D050001E4691465FEA010809D046B138B1044640
:10D0600006F035FE002803D100250B4F10E00E20FE
:10D07000BDE8F88305EB850004EB400033464A46E3
:10D080004146801C009704F0CFFA0028F0D16D1CB7
:10D090002188A942EED8EBE711CC01002DE9FE432F
:10D0A0001D461646040007D036B12DB1208835281C
:10D0B00004D00720BDE8FE830E20FBE7002001908E
:10D0C0002F6835200DF10408ADF8080043463A46B4
:10D0D000314602A806F0FBFD0028EBD143463A4654
:10D0E0003146201D06F0F3FD0028E3D143463A46C1
:10D0F0003146A01D06F0EBFD0028DBD143463A4641
:10D10000314604F1080006F0E2FD0028D2D10748BC
:10D11000009043463A46314604F10A0004F07AFA98
:10D120000028C7D101992960C4E7000031D101006E
:10D13000F8B51D4617460E001AD0CDB1C0B1044651
:10D1400006F0C5FD002812D12B463A463146A01CF8
:10D1500006F0BDFD00280AD160882188801C484364
:10D1600081B23B463246201D009506F032FEF8BDE6
:10D170000E20F8BD2DE9FE431D461646040007D0DB
:10D1800036B12DB12088372804D00720BDE8FE83B2
:10D190000E20FBE7002001902F6837200DF10408D6
:10D1A000ADF8080043463A46314602A806F08FFD26
:10D1B0000028EBD143463A463146201D06F087FD54
:10D1C0000028E3D143463A463146A01D06F07FFDD4
:10D1D0000028DBD143463A46314604F1080006F008
:10D1E00076FD0028D2D10748009043463A463146A2
:10D1F00004F10A0004F00EFA0028C7D10199296051
:10D20000C4E7000009D20100F8B51D4617460E001C
:10D210000ED06DB160B1044606F059FD002806D16C
:10D22000009521883B463246A01C06F0D2FDF8BD91
:10D230000E20F8BD2DE9FE431D461646040007D01A
:10D2400036B12DB12088332804D00720BDE8FE83F5
:10D250000E20FBE7002001902F6833200DF1040819
:10D26000ADF8080043463A46314602A806F02FFDC5
:10D270000028EBD143463A463146201D06F027FDF3
:10D280000028E3D143463A463146A01D06F01FFD73
:10D290000028DBD143463A46314604F1080006F047
:10D2A00016FD0028D2D10748009043463A46314641
:10D2B00004F10A0004F0AEF90028C7D101992960F1
:10D2C000C4E70000C9D201002DE9F8431E4691468B
:10D2D0005FEA010809D046B138B1044606F0F7FC10
:10D2E000002803D100250B4F10E00E20BDE8F88385
:10D2F00005EB450004EB400033464A464146801C9E
:10D30000009704F091F90028F0D16D1C2188A94202
:10D31000EED8EBE70DCE01002DE9FE431D46164683
:10D32000040007D036B12DB120883A2804D0072058
:10D33000BDE8FE830E20FBE7002001902F683A2015
:10D340000DF10408ADF8080043463A46314602A8FC
:10D3500006F0BDFC0028EBD143463A463146201D7D
:10D3600006F0B5FC0028E3D143463A463146A01DFD
:10D3700006F0ADFC0028DBD143463A46314604F1C5
:10D38000080006F0A4FC0028D2D1074800904346CC
:10D390003A46314604F10A0004F03CF90028C7D1AE
:10D3A00001992960C4E70000ADD3010019B113B1A0
:10D3B00008B106F08CBC0E20704700002DE9FE433A
:10D3C0001D461646040007D036B12DB120883928F5
:10D3D00004D00720BDE8FE830E20FBE7002001906B
:10D3E0002F6839200DF10408ADF8080043463A468D
:10D3F000314602A806F06BFC0028EBD143463A46C2
:10D400003146201D06F063FC0028E3D143463A462E
:10D410003146A01D06F05BFC0028DBD143463A46AE
:10D42000314604F1080006F052FC0028D2D107482A
:10D43000009043463A46314604F10A0004F0EAF807
:10D440000028C7D101992960C4E7000051D4010028
:10D45000F8B51D4617460E001ED0EDB1E0B10446EA
:10D4600006F035FC002816D12B463A463146A01C62
:10D4700006F08CFC00280ED12B463A463146201D82
:10D4800006F025FC002806D10095A1883B463246CF
:10D49000A01D06F09EFCF8BD0E20F8BD2DE9FE4350
:10D4A0001D461646040007D036B12DB1208830281D
:10D4B00004D00720BDE8FE830E20FBE7002001908A
:10D4C0002F6830200DF10408ADF8080043463A46B5
:10D4D000314602A806F0FBFB0028EBD143463A4652
:10D4E0003146201D06F0F3FB0028E3D143463A46BF
:10D4F0003146A01D06F0EBFB0028DBD143463A463F
:10D50000314604F1080006F0E2FB0028D2D10748BA
:10D51000009043463A46314604F10A0004F07AF896
:10D520000028C7D101992960C4E7000031D5010066
:10D530002DE9F8431E4691465FEA010809D046B13D
:10D5400038B1044606F0C3FB002803D100250A4F7A
:10D550000EE00E20BDE8F88304EBC50033464A46D2
:10D560004146801C009704F05FF80028F2D16D1C42
:10D570002188A942F0D8EDE709DC01002DE9FE433E
:10D580001D461646040007D036B12DB12088362836
:10D5900004D00720BDE8FE830E20FBE700200190A9
:10D5A0002F6836200DF10408ADF8080043463A46CE
:10D5B000314602A806F08BFB0028EBD143463A46E1
:10D5C0003146201D06F083FB0028E3D143463A464E
:10D5D0003146A01D06F07BFB0028DBD143463A46CE
:10D5E000314604F1080006F072FB0028D2D107484A
:10D5F000009043463A46314604F10A0004F00AF826
:10D600000028C7D101992960C4E7000011D60100A4
:10D61000F8B51D4617460E001ED0EDB1E0B1044628
:10D6200006F055FB002816D12B463A463146A01C81
:10D6300006F04DFB00280ED12B463A463146201D00
:10D6400006F045FB002806D10095A1883B463246EE
:10D65000A01D06F0BEFBF8BD0E20F8BD2DE9FE436F
:10D660001D461646040007D036B12DB1208831285A
:10D6700004D00720BDE8FE830E20FBE700200190C8
:10D680002F6831200DF10408ADF8080043463A46F2
:10D69000314602A806F01BFB0028EBD143463A4670
:10D6A0003146201D06F013FB0028E3D143463A46DD
:10D6B0003146A01D06F00BFB0028DBD143463A465D
:10D6C000314604F1080006F002FB0028D2D10748D9
:10D6D000009043463A46314604F10A0003F09AFFAF
:10D6E0000028C7D101992960C4E70000F1D60100E4
:10D6F0002DE9F84F984692465FEA01090ED0B8F13D
:10D70000000F0BD050B104464346494606F0DFFAFD
:10D71000002804D1A51C0026094F0DE00E20BDE80D
:10D72000F88F4346524649462846009703F07CFF4F
:10D730000028F4D10A35761C2188B142F1D8EEE7F1
:10D740007DDA01002DE9FE431D461646040007D090
:10D7500036B12DB120883B2804D00720BDE8FE83D8
:10D760000E20FBE7002001902F683B200DF10408FC
:10D77000ADF8080043463A46314602A806F0A7FA3B
:10D780000028EBD143463A463146201D06F09FFA69
:10D790000028E3D143463A463146A01D06F097FAE9
:10D7A0000028DBD143463A46314604F1080006F032
:10D7B0008EFA0028D2D10748009043463A463146B7
:10D7C00004F10A0003F026FF0028C7D1019929605F
:10D7D000C4E70000D9D7010019B113B108B106F0B0
:10D7E000D5BA0E2070472DE9FC411D4616460400AF
:10D7F00007D036B12DB120883C2804D00720BDE8E1
:10D80000FC810E20FBE7002000902F683C20E846BA
:10D81000ADF8040043463A46314601A806F057FAEF
:10D820000028ECD143463A463146201D06F04FFA17
:10D830000028E4D143463A463146A01D06F047FA97
:10D840000028DCD143463A46314604F1080006F090
:10D850003EFA0028D3D143463A46314604F10A0045
:10D8600006F094FA0028CAD100992960C7E70000A1
:10D870002DE9FE431D461646040007D036B12DB1F2
:10D880002088382804D00720BDE8FE830E20FBE75F
:10D89000002001902F6838200DF10408ADF8080031
:10D8A00043463A46314602A806F011FA0028EBD169
:10D8B00043463A463146201D06F009FA0028E3D1D6
:10D8C00043463A463146A01D06F001FA0028DBD156
:10D8D00043463A46314604F1080006F0F8F90028BC
:10D8E000D2D10748009043463A46314604F10A0037
:10D8F00003F090FE0028C7D101992960C4E7000019
:10D9000005D90100F8B51D4617460E0027D035B3DE
:10D9100028B3044606F0DBF900281FD12B463A460F
:10D920003146A01C06F032FA002817D12B463A46A1
:10D930003146201D06F0CBF900280FD12B463A4680
:10D940003146A01D06F0C3F9002807D10095E188F3
:10D950003B46324604F1080006F03BFAF8BD0E20C3
:10D96000F8BDF8B51F460C46050008D02CB10020C4
:10D97000009028786E46A52803D00720F8BD0E2019
:10D98000F8BD0120134600903246284606F090F973
:10D990000028F5D13B4632462146284606F088F954
:10D9A0000028EDD10098A04201D00920F8BD002048
:10D9B000F8BD13460A460146A52005F0ADB92DE98C
:10D9C000F041164607000FD076B16BB11C460D46EC
:10D9D00006F06EF9002808D1A31C324629463846C5
:10D9E000BDE8F04106F064B90E20BDE8F0812DE9F4
:10D9F000F0411D4617460E000ED06DB160B10446D1
:10DA000006F065F9002808D12B463A463146A01C9D
:10DA1000BDE8F04106F05BB90E20BDE8F081F8B535
:10DA20001F460C46050008D02CB100200090287835
:10DA30006E46A42803D00720F8BD0E20F8BD0120B3
:10DA4000134600903246284606F032F90028F5D1F8
:10DA50003B4632462146284606F02AF90028EDD1F9
:10DA60000098A04201D00920F8BD0020F8BD13465F
:10DA70000A460146A42005F04FB90000F8B51D463E
:10DA800017460E000FD075B168B1044606F01FF9B5
:10DA9000002807D1054800902B463A463146A01C85
:10DAA00003F0C2FDF8BD0E20F8BD000009DC010046
:10DAB0002DE9FC411F46DDF820800C46050009D009
:10DAC0002CB100200190287801AE9B2804D00720BB
:10DAD000BDE8FC810E20FBE7012013460190324691
:10DAE000284606F0E5F80028F2D13B4632462146AA
:10DAF000284606F0DDF80028EAD1084800904346A1
:10DB000032462146284601F0F9FF0028E0D101986D
:10DB1000A04201D00920DBE70020D9E7C1F60100CF
:10DB200013460A4601469B2005F0F6B82DE9F84356
:10DB30001F46DDF820800C46050009D02CB10020DE
:10DB4000009028786E46A12804D00720BDE8F8830D
:10DB50000E20FBE70120134600903246284606F0CF
:10DB6000A7F80028F2D13B4632462146284606F067
:10DB70009FF80028EAD1434632462146284606F05F
:10DB800097F80028E2D10098A04201D00920DDE7F3
:10DB90000020DBE713460A460146A12005F0BCB889
:10DBA0002DE9FC411F460C46050009D02CB1002090
:10DBB0000190287801AE9C2804D00720BDE8FC81A4
:10DBC0000E20FBE70120134601903246284606F05E
:10DBD0006FF80028F2D1084800903B4632462146B3
:10DBE000284601F08BFF0028E8D10198A04201D01F
:10DBF0000920E3E70020E1E7BFD9010013460A4608
:10DC000001469C2005F088B8F8B51D4617460E0061
:10DC100012D08DB180B1044608480090204603F030
:10DC200003FD002807D1064800902B463A463146AE
:10DC3000201D03F0F9FCF8BD0E20F8BDF1F601003F
:10DC4000EFD90100F8B51646070028D03EB333B32C
:10DC50001C460D4606F08DF800281FD1631C324685
:10DC60002946384606F085F8002817D1A31C32460D
:10DC70002946384606F01CF800280FD1231D3246ED
:10DC80002946384606F014F8002807D1A01D831C49
:10DC9000009032462946384604F007F8F8BD0E20B9
:10DCA000F8BD00002DE9FC411F460C46050009D0D7
:10DCB0002CB100200190287801AEA32804D00720C1
:10DCC000BDE8FC810E20FBE701201346019032469F
:10DCD000284605F0EDFF0028F2D1084800903B46A9
:10DCE00032462146284601F009FF0028E8D1019874
:10DCF000A04201D00920E3E70020E1E745DC010074
:10DD000013460A460146A32005F006B82DE9FC4754
:10DD10009846DDF828900D46060009D02DB1002464
:10DD20000194307801AFB42804D00720BDE8FC8707
:10DD30000E20FBE70120134601903A46304605F0DD
:10DD4000B7FF0028F2D143463A46294630460094B0
:10DD500001F0D4FE0028E9D14B463A462946304628
:10DD6000009401F0CBFE0028E0D10198A84201D038
:10DD70000920DBE70020D9E72DE9FF4383B098466F
:10DD8000DDF8389014460F0019D0C4B1002001907E
:10DD90002568B42001AE8DF8080033462A4602A853
:10DDA00005F0F4FF00280BD133462A46394603A874
:10DDB00005F0BEFF002803D10398C0B903E00E2090
:10DDC00007B0BDE8F0830C48009033462A46394638
:10DDD000404601F0C1FE0028F2D1084800903346C9
:10DDE0002A463946484601F0B7FE0028E8D1019896
:10DDF00020600020E4E70000F1F601006DDE010084
:10DE00002DE9FC4116465FEA00082BD056B34BB310
:10DE1000154F1C460D46009703F0CAFB00281FD182
:10DE2000631C324629464046009703F0C1FB002898
:10DE300016D101AB32462946404605F09AFF00282C
:10DE40000ED19DF80410A2784B0861F3000263F331
:10DE50004202CB0863F3C302090961F30412A27002
:10DE6000BDE8FC810E20FBE7D1A901002DE9FC41B2
:10DE70001D4690460E0032D085B378B3194F044644
:10DE8000009703F0E5FB002826D12B464246314699
:10DE9000601C009703F0DCFB00281DD1A0782B4606
:10DEA000C0F34102014662F35F01C0F3C00241EAE0
:10DEB000C201C0F3001041EA00108DF80400424690
:10DEC000314601A805F062FF002805D1A178C1F311
:10DED0004101012900D00720BDE8FC81FFE70E20A9
:10DEE000FAE7000003AA0100F8B51646070032D091
:10DEF00086B37BB3194800901C460D46384601F0A6
:10DF0000FDFD002825D116480090231D32462946E4
:10DF1000384601F0F3FD00281BD104F10A03324614
:10DF20002946384605F0C4FE002812D104F10C033E
:10DF300032462946384605F0BBFE002809D104F1D7
:10DF40000800009004F1100332462946384603F0D9
:10DF5000ACFEF8BDFFE70E20FBE70000C1F60100B4
:10DF600001DE01002DE9FC411646070028D03EB332
:10DF700033B31C460D4605F09BFE00281ED101ABB5
:10DF800032462946384605F0F4FE002816D1231DF6
:10DF900032462946384605F08BFE00280ED1A01DDA
:10DFA000831C009032462946384603F07EFE002846
:10DFB00004D19DF8041001F00101A170BDE8FC81BD
:10DFC0000E20FBE718B112B10BB105F09ABE0E207E
:10DFD000704738B558B152B14BB11C466B4605F08D
:10DFE000C8FE002802D19DF80010217038BD0E2017
:10DFF00038BD2DE9F0411D4617460E001ED0EDB18B
:10E00000E0B1044605F063FE002818D12B463A46DD
:10E010003146A01C05F05BFE002810D12B463A4685
:10E020003146201D05F053FE002808D12B463A4604
:10E030003146A01DBDE8F04105F049BE0E20BDE807
:10E04000F08100002DE9F84316465FEA000854D03D
:10E05000002E52D0002B50D0294800901C460D466F
:10E06000404603F0A5FA002845D126480090631CDD
:10E0700032462946404603F09BFA00283BD104F182
:10E08000080332462946404605F012FE002832D1E8
:10E0900004F10A000090231D32462946404603F051
:10E0A00004FE002827D11848009004F10C033246E2
:10E0B0002946404601F022FD00281CD1134F04F1EF
:10E0C0001003324629464046009701F017FD00280C
:10E0D00011D104F11403324629464046009701F05D
:10E0E0000DFD002807D104F11803324629464046A9
:10E0F000009701F003FDBDE8F8830E20FBE7000068
:10E100006FCA01003DCA010011E1010001DE0100FA
:10E110002DE9F0411646070027D036B32BB31C4635
:10E120000D4605F026FE002820D1631C3246294604
:10E13000384605F01EFE002818D1A31C3246294699
:10E14000384605F0B5FD002810D1231D324629467A
:10E15000384605F00EFE002808D1A31D3246294698
:10E160003846BDE8F04105F0A3BD0E20BDE8F081C2
:10E170002DE9FC479846DDE90A9A0C46050009D0CE
:10E180002CB100260196287801AFAA2804D00720D8
:10E19000BDE8FC870E20FBE70120134601903A46BC
:10E1A000284605F085FD0028F2D11248009043462C
:10E1B0003A462146284601F0A1FC0028E8D10E4845
:10E1C00000904B463A462146284601F097FC00282D
:10E1D000DED153463A4621462846009601F08EFC91
:10E1E0000028D5D10198A04201D00920D0E7002015
:10E1F000CEE7000045E00100E9DE01002DE9FF4126
:10E2000084B0984614460F0019D0C4B10020019084
:10E210002568AA2001AE8DF8080033462A4602A8D8
:10E2200005F0B4FD00280BD133462A46394604A830
:10E2300005F07EFD002803D1049870B903E00E209C
:10E2400008B0BDE8F0810748009033462A463946B9
:10E25000404601F081FC0028F2D1019820600020A6
:10E26000EEE70000F3DF010018B112B10BB105F0C9
:10E2700080BD0E20704700002DE9FC479846DDF870
:10E2800028900C46050009D02CB10026019628786C
:10E2900001AFAB2804D00720BDE8FC870E20FBE7C8
:10E2A0000120134601903A46284605F001FD00285A
:10E2B000F2D10D48009043463A462146284601F0E7
:10E2C0001DFC0028E8D14B463A46214628460096D8
:10E2D00001F014FC0028DFD10198A04201D00920F0
:10E2E000DAE70020D8E70000E9DE01002DE9FF4170
:10E2F00084B0984614460F0019D0C4B10020019094
:10E300002568AB2001AE8DF8080033462A4602A8E6
:10E3100005F03CFD00280BD133462A46394604A8B7
:10E3200005F006FD002803D1049870B903E00E2023
:10E3300008B0BDE8F0810748009033462A463946C8
:10E34000404601F009FC0028F2D10198206000202D
:10E35000EEE70000CF3C02002DE9FE431D461646C5
:10E36000040007D036B12DB12088552804D00720ED
:10E37000BDE8FE830E20FBE7002001902F685520AA
:10E380000DF10408ADF8080043463A46314602A8AC
:10E3900005F09DFC0028EBD143463A463146201D4E
:10E3A00005F095FC0028E3D10648009043463A4624
:10E3B0003146A01D03F042F90028D9D10199296006
:10E3C000D6E70000C9E3010019B113B108B105F0A7
:10E3D0007EBC0E20704700002DE9FE431D46164608
:10E3E000040007D036B12DB12088532804D007206F
:10E3F000BDE8FE830E20FBE7002001902F6853202C
:10E400000DF10408ADF8080043463A46314602A82B
:10E4100005F05DFC0028EBD143463A463146201D0D
:10E4200005F055FC0028E3D10648009043463A46E3
:10E430003146A01D03F002F90028D9D101992960C5
:10E44000D6E7000049E4010019B113B108B105F0A5
:10E450003EBC0E2070472DE9FC411D4616460400C7
:10E4600007D036B12DB12088572804D00720BDE849
:10E47000FC810E20FBE7002000902F685720E84623
:10E48000ADF8040043463A46314601A805F01FFCAA
:10E490000028ECD143463A463146201D05F017FCD2
:10E4A0000028E4D143463A463146A01D05F06EFCF3
:10E4B0000028DCD100992960D9E70000F8B51D4695
:10E4C00017460E0019D0C5B1B8B1044605F0FFFBE0
:10E4D000002813D10A4800902B463A463146A01C2A
:10E4E00003F0B6F8002809D101B02B463A46314670
:10E4F000A01DBDE8F04005F0EABB0E20F8BD00000D
:10E50000F1F601002DE9F04186B01E4617460400E1
:10E5100008D03FB136B12088512805D0072006B079
:10E52000BDE8F0810E20FAE7002003903568512005
:10E530000DF10C08ADF8100043462A46394604A8F0
:10E5400005F0C5FB0028EAD143462A463946201D7E
:10E5500005F0BDFB0028E2D11648009043462A464C
:10E560003946A01D03F06AF80500D8D1A079022829
:10E570001CD1A07B062801D0042817D1A08801A9AE
:10E5800001F0C8FB052811D003A80090019833685A
:10E5900000EB400101EB001107483A4600EB810017
:10E5A0000189406803F099FB0500B8D103983060F9
:10E5B0002846B4E7BDE50100A8460020F8B51D4691
:10E5C00017460E000DD065B158B1044605F0DEFBCC
:10E5D000002805D12078012805D0022805D0072081
:10E5E000F8BD0E20F8BD054800E0054800902B4618
:10E5F0003A463146A01C03F02BF8F8BDBDE40100FB
:10E600000DE801002DE9FC411C461646050007D027
:10E6100036B12CB12888532804D00720BDE8FC81EE
:10E620000E20FBE70020009027685320E846ADF855
:10E63000040043463A46314601A805F048FB00284D
:10E64000ECD143463A463146281D05F040FB0028F0
:10E65000E4D100992160E1E72DE9FE431D4616460D
:10E66000040007D036B12DB12088522804D00720ED
:10E67000BDE8FE830E20FBE7002001902F685220AA
:10E680000DF10408ADF8080043463A46314602A8A9
:10E6900005F01DFB0028EBD143463A463146201DCC
:10E6A00005F015FB0028E3D10648009043463A46A2
:10E6B0003146A01D02F0C2FF0028D9D1019929607E
:10E6C000D6E70000C9E6010019B113B108B105F0A1
:10E6D0005DBB0E20704700002DE9FE431D46164627
:10E6E000040007D036B12DB12088562804D0072069
:10E6F000BDE8FE830E20FBE7002001902F68562026
:10E700000DF10408ADF8080043463A46314602A828
:10E7100005F0DDFA0028EBD143463A463146201D8C
:10E7200005F0D5FA0028E3D10648009043463A4662
:10E730003146A01D02F082FF0028D9D1019929603D
:10E74000D6E7000049E7010019B113B108B105F09F
:10E750001DBB0E20704700002DE9FF471E46914665
:10E7600004000AD0B9F1000F07D036B12088502834
:10E7700005D0072004B0BDE8F0870E20FAE700209E
:10E780000190D6F80080502001AFADF808003B465C
:10E790004246494602A805F09AFA0028EAD13B46CB
:10E7A00042464946201D05F092FA0028E2D115485C
:10E7B00000903B4642464946A01D02F03FFF05003F
:10E7C000D8D1207B012801D0062816D1A08803A922
:10E7D00001F0A0FA052810D00398009700EB400143
:10E7E00001EB00110848434600EB81004A460189CD
:10E7F000406803F072FA0500BCD1019830602846E9
:10E80000B8E700000DE80100A8460020F8B51D4655
:10E8100017460E003CD0D5B3C8B3044605F057FAEE
:10E82000002833D11B4800902B463A463146A01CA5
:10E8300002F00EFF002829D12B463A463146A01D92
:10E8400005F0A4FA002821D12B463A463146E01DB6
:10E8500005F09CFA002819D12B463A46314604F1BE
:10E86000080005F034FA002810D12B463A4631460C
:10E8700004F10A0005F02BFA002807D10095618900
:10E880003B46324604F10C0005F0A3FAF8BDFFE761
:10E890000E20FBE7F1F60100F8B51F460C46050017
:10E8A00008D02CB10020009028786E46B52803D0FF
:10E8B0000720F8BD0E20F8BD012013460090324617
:10E8C000284605F0F5F90028F5D13B4632462146A9
:10E8D000284605F0EDF90028EDD10098A04201D0BE
:10E8E0000920F8BD0020F8BD13460A460146B520B0
:10E8F00004F012BA2DE9FC411646070032D086B367
:10E900007BB31C460D4605F0D3F9002827D1A31C84
:10E9100032462946384605F02CFA00281FD1231D1F
:10E9200032462946384605F0C3F9002817D10E486B
:10E93000009004F1080332462946384601F0DEF81B
:10E9400000280CD1A168002909D008880090019006
:10E9500004F10C0332462946384600F0C5FFBDE8F5
:10E96000FC81FFE70E20FAE7B13C02002DE9FC41F3
:10E970001F460C46050009D02CB1002001902878D4
:10E9800001AEAE2804D00720BDE8FC810E20FBE7D5
:10E990000120134601903246284605F089F90028E7
:10E9A000F2D1084800903B4632462146284601F005
:10E9B000A5F80028E8D10198A04201D00920E3E79A
:10E9C0000020E1E7F5E801002DE9FF4184B0984619
:10E9D00014460F0019D0C4B1002001902568AE2064
:10E9E00001AE8DF8080033462A4602A805F0CEF99C
:10E9F00000280BD133462A46394604A805F098F979
:10EA0000002803D1049870B903E00E2008B0BDE8D7
:10EA1000F0810748009033462A463946404601F0C7
:10EA20009BF80028F2D1019820600020EEE700005A
:10EA3000CF3C02002DE9FC479846DDF828900C46B3
:10EA4000050009D02CB100260196287801AFA9282D
:10EA500004D00720BDE8FC870E20FBE70120134609
:10EA600001903A46284605F023F90028F2D14346A2
:10EA70003A462146284605F01BF90028EAD14B46C4
:10EA80003A4621462846009601F038F80028E1D1A0
:10EA90000198A04201D00920DCE70020DAE700005D
:10EAA0002DE9FF4184B0984614460F0019D0C4B137
:10EAB000002001902568A92001AE8DF8080033469A
:10EAC0002A4602A805F062F900280BD133462A46EF
:10EAD000394604A805F02CF9002803D1049870B930
:10EAE00003E00E2008B0BDE8F081074800903346EF
:10EAF0002A463946404601F02FF80028F2D1019805
:10EB000020600020EEE70000CF3C02007CB50C4600
:10EB100040B12CB100230193057801A9B32D03D096
:10EB200007207CBD0E207CBD0125CDE900351346B4
:10EB30000A46214600F0E2FF0028F4D10198A042E5
:10EB400001D009207CBD00207CBD00002DE9FF41E3
:10EB500084B0984614460F0019D0C4B1002001902B
:10EB60002568B32001AE8DF8080033462A4602A876
:10EB700005F00CF900280BD133462A46394604A883
:10EB800005F0D6F8002803D1049870B903E00E20F0
:10EB900008B0BDE8F0810748009033462A46394660
:10EBA000404600F0D9FF0028F2D1019820600020F3
:10EBB000EEE70000CF3C0200F8B5164607000FD084
:10EBC00076B16BB11C460D4605F0D3F8002806D18E
:10EBD00020780849012805D0022803D00720F8BD75
:10EBE0000E20F8BD0091231D32462946384602F01A
:10EBF000DFFCF8BD65DF01002DE9FC411F460C4636
:10EC0000050009D02CB100200190287801AEB02871
:10EC100004D00720BDE8FC810E20FBE7012013464D
:10EC200001903246284605F043F80028F2D1084802
:10EC300000903B4632462146284600F05FFF002800
:10EC4000E8D10198A04201D00920E3E70020E1E7E4
:10EC5000B9EB010013460A460146B02004F05CB847
:10EC60002DE9FC479846DDF828900C46050009D0B0
:10EC70002CB100260196287801AFA82804D00720DF
:10EC8000BDE8FC870E20FBE70120134601903A46C1
:10EC9000284605F06EF80028F2D10D480090434652
:10ECA0003A462146284600F029FF0028E8D14B4685
:10ECB0003A4621462846009600F020FF0028DFD182
:10ECC0000198A04201D00920DAE70020D8E700002F
:10ECD000C1F601002DE9FF4184B0984614460F00AB
:10ECE00019D0C4B1002001902568A82001AE8DF88C
:10ECF000080033462A4602A805F048F800280BD140
:10ED000033462A46394604A805F012F8002803D1F4
:10ED1000049870B903E00E2008B0BDE8F081074800
:10ED2000009033462A463946404600F015FF002839
:10ED3000F2D1019820600020EEE70000CF3C0200F5
:10ED40002DE9F8431F46DDF820800C46050009D068
:10ED50002CB10020009028786E46AF2804D0072000
:10ED6000BDE8F8830E20FBE70120134600903246F1
:10ED7000284604F09DFF0028F2D13B46324621464A
:10ED8000284604F095FF0028EAD143463246214642
:10ED9000284604F08DFF0028E2D10098A04201D05F
:10EDA0000920DDE70020DBE713460A460146AF20D5
:10EDB00003F0B2BF2DE9FC479946DDE90A8A0C460B
:10EDC000050009D02CB100260196287801AFB228A1
:10EDD00004D00720BDE8FC870E20FBE70120134686
:10EDE00001903A46284604F063FF0028F2D111480A
:10EDF000009043463A462146284600F07FFE002810
:10EE0000E8D14B463A4621462846009600F076FE69
:10EE10000028DFD153463A462146284604F071FFC8
:10EE20000028D7D10198A04201D00920D2E70020C4
:10EE3000D0E70000B13C02002DE9FF4383B09946C2
:10EE40000E9E14465FEA01081AD0CCB10020019052
:10EE50002768B22001AD8DF808002B463A4641469E
:10EE600002A804F093FF00280BD12B463A464146F6
:10EE700003A804F05DFF002803D10398C0B903E0A4
:10EE80000E2007B0BDE8F0830B4800902B463A46B1
:10EE90004146304600F060FE0028F2D146B10095B0
:10EEA00031883B464246484600F050FD0028E8D1F4
:10EEB000019820600020E4E7CF3C02002DE9FC47E8
:10EEC0009846DDE90A790C46050009D02CB10020EE
:10EED0000190287801AEB12804D00720BDE8FC8756
:10EEE0000E20FBE70120134601903246284604F02D
:10EEF000DFFE0028F2D143463246214628460097DD
:10EF000002F0D3FE0028E9D14B463246214628467E
:10EF100004F0F7FE0028E1D10198A04201D00920B9
:10EF2000DCE70020DAE713460A460146B12003F089
:10EF3000F3BE2DE9FC4799460A9D0E4607000AD00C
:10EF400036B10024019438780DF10408AD2804D0BE
:10EF50000720BDE8FC870E20FBE701201346019047
:10EF60004246384604F0A4FE0028F2D14B46424601
:10EF70003146384604F09CFE0028EAD12B46424632
:10EF800031463846009400F0B9FD0028E1D12B68E5
:10EF9000CBB14246314638469B1C04F089FE00281E
:10EFA000D7D14246314638462B6804F081FE00280E
:10EFB000CFD12B684246314638461B1D009400F0E5
:10EFC0009DFD0028C5D10198B04201D00920C0E7BD
:10EFD0000020BEE72DE9FF4184B0984614460F009B
:10EFE00019D0C4B1002001902568AD2001AE8DF884
:10EFF000080033462A4602A804F0C8FE00280BD1B8
:10F0000033462A46394604A804F092FE002803D16C
:10F01000049870B903E00E2008B0BDE8F0810748FD
:10F02000009033462A463946404600F095FD0028B8
:10F03000F2D1019820600020EEE700004BF10100C2
:10F040002DE9FC411F46DDF820800C46050009D063
:10F050002CB100200190287801AEAC2804D0072004
:10F06000BDE8FC810E20FBE70120134601903246EB
:10F07000284604F01DFE0028F2D13B4632462146C8
:10F08000284604F015FE0028EAD1084800904346BF
:10F0900032462146284600F031FD0028E0D1019893
:10F0A000A04201D00920DBE70020D9E71DF10100D3
:10F0B0002DE9FF4184B0984614460F0019D0C4B121
:10F0C000002001902568AC2001AE8DF80800334681
:10F0D0002A4602A804F05AFE00280BD133462A46DD
:10F0E000394604A804F024FE002803D1049870B91E
:10F0F00003E00E2008B0BDE8F081074800903346D9
:10F100002A463946404600F027FD0028F2D10198F2
:10F1100020600020EEE700004BF10100F8B5164634
:10F12000070010D07EB173B11C460D469B1C04F045
:10F13000BFFD002806D1324629463846231D0094DB
:10F1400002F0B3FDF8BD0E20F8BDF8B51D46174618
:10F150000E000FD075B168B10446801C04F0B7FDF5
:10F16000002806D1009521883B463246606802F0AF
:10F17000B4FDF8BD0E20F8BD2DE9FC411C460D463E
:10F18000060025D035B10027019730780DF104082D
:10F19000682802D00720BDE8FC8101200190BAB1A7
:10F1A000B4B12068A0B113464246304604F0A9FD30
:10F1B0000028F0D12346424629463046009700F009
:10F1C0009DFC0028E7D10198A84203D00920E2E77E
:10F1D0000E20E0E70020DEE72DE9FF4184B0154670
:10F1E0000E9C5FEA01082FD075B3002001902E68B5
:10F1F000682001AF8DF808003B463246414602A820
:10F2000004F0C4FD002820D13B463246414604A804
:10F2100004F08EFD002818D1049850BBA4B13B46E1
:10F220003246414607A804F083FD00280DD1002195
:10F23000079A0846212A22D00ADC012A0DD0022A88
:10F240000DD0202A0DD118E00E2008B0BDE8F081C5
:10F25000222A16D0242A04D115E00C4900E00C49DA
:10F26000204600913B463246414602F0B5F900285F
:10F27000EBD1019828600020E7E70649F0E706494E
:10F28000EEE70649ECE70649EAE70000959C010035
:10F29000079C01005DBD0100CDBD010029BE01003C
:10F2A000FFBC010038B580B129B100230093037879
:10F2B0006C46672B01D0072038BD0123009322B193
:10F2C0001346224604F01DFD38BD0E2038BD000057
:10F2D0002DE9FC471F46060014460D4631D045B1C6
:10F2E0004FF00008CDF8048030780DF1040967284C
:10F2F00002D00720BDE8FC87012001900CB307B3C2
:10F300003868F0B113464A46304604F0FAFC00284B
:10F31000F0D13B464A4629463046CDF8008000F001
:10F32000EDFB0028E6D1396801B322680346212AA3
:10F3300023D008DC012A0DD0022A0DD0202A0DD1BD
:10F3400019E00E20D6E7222A19D0242A19D0252A1E
:10F3500004D118E00E4800E00E480B4600904A46E3
:10F360002946304602F010F90028C3D10198A8427E
:10F370000BD00920BEE70848EFE70848EDE708484A
:10F38000EBE70848E9E70848E7E70020B2E70000B4
:10F39000259C0100E39B01002FBD010089BD0100F8
:10F3A00011BE0100CFBC010045BE010013460A4654
:10F3B0000146672003F0B0BC38B5D0B1CAB1C3B1C3
:10F3C0001C466B4604F0D5FC002811D19DF80020A6
:10F3D000217862F3000121709DF80020520862F349
:10F3E000410121709DF80020920862F3870121708D
:10F3F00038BD0E2038BD38B581B17BB170B1007811
:10F40000C0F34005044665F35F0420F003000443A5
:10F410008DF80040684604F0B9FC38BD0E2038BDB8
:10F42000F8B51546060010D07DB173B11F460C46E5
:10F430001B1D04F03DFC002806D100903B462A46E7
:10F440002146304600F05AFBF8BD0E20F8BD000002
:10F450002DE9FC411C460D46060025D02DB10020AB
:10F460000190307801AF662802D00720BDE8FC810A
:10F4700001200190C2B1BCB12068A8B113463A4640
:10F48000304604F015FC0028F0D1094800902346CE
:10F490003A462946304600F031FB0028E6D1019873
:10F4A000A84203D00920E1E70E20DFE70020DDE7D6
:10F4B00021F4010013460A460146662003F02CBCE5
:10F4C00038B530B12AB123B11024009404F06BFC9C
:10F4D00038BD0E2038BD08B541B13BB130B1009305
:10F4E00013460A46102104F074FC08BD0E2008BD26
:10F4F0002DE9FC410C46DDF82080050009D02CB137
:10F5000000260196287801AF632804D00720BDE8C3
:10F51000FC810E20FBE70120CDE900203A46284679
:10F5200002F0F3FB0028F2D143463A462146284632
:10F53000009600F0E3FA0028E9D10198A04201D03A
:10F540000920E4E70020E2E72DE9FF4184B0984676
:10F5500014460F0019D0C4B1002001902568632023
:10F5600001AE8DF8080033462A4602A804F00EFCCE
:10F5700000280BD133462A46394604A804F0D8FBAC
:10F58000002803D1049870B903E00E2008B0BDE84C
:10F59000F0810748009033462A463946404600F03D
:10F5A000DBFA0028F2D1019820600020EEE700008D
:10F5B000F1F601002DE9FC471D460A9C0E460700A6
:10F5C00039D046B14FF00008CDF8048038780DF1FD
:10F5D0000409642802D00720BDE8FC8701200190BF
:10F5E0004AB345B33CB3106828B3286818B3206801
:10F5F00008B31348134600904A46384600F07EFA96
:10F600000028E9D12B464A4631463846CDF80080DD
:10F6100000F074FA0028DFD123464A4631463846C6
:10F62000CDF8008000F06AFA0028D5D10198B042E8
:10F6300003D00920D0E70E20CEE70020CCE7000061
:10F64000C1F601002DE9FF4184B01446DDF8388091
:10F650000F0019D0C4B1002001902668642001ADCC
:10F660008DF808002B46324602A804F08FFB0028D4
:10F670000BD12B463246394604A804F059FB00282A
:10F6800003D10498C0B903E00E2008B0BDE8F081B2
:10F690002B463246394607A804F078FB0028F4D1FF
:10F6A000B8F1000008D033463A4600959DF81C108A
:10F6B00004F08FFB0028E8D1019820600020E4E7E7
:10F6C0002DE9F041164607000FD076B16BB11C460C
:10F6D0000D4604F0EDFA002808D1A31C3246294655
:10F6E0003846BDE8F04104F044BB0E20BDE8F0818F
:10F6F0002DE9F0411D4617460E000ED06DB160B1E8
:10F70000044604F0E4FA002808D12B463A46314674
:10F71000A01CBDE8F04104F039BB0E20BDE8F0812B
:10F720002DE9FC411C460D46060029D035B10027C5
:10F73000019730780DF10408622802D00720BDE857
:10F74000FC8101200190DAB1D4B11068C0B1206809
:10F75000B0B10D48134600904246304600F0CEF955
:10F760000028ECD12346424629463046009700F057
:10F77000C5F90028E3D10198A84203D00920DEE7AB
:10F780000E20DCE70020DAE7C1F401002DE9FF419B
:10F7900084B0984614460F0019D0C4B100200190DF
:10F7A0002568622001AE8DF8080033462A4602A87B
:10F7B00004F0ECFA00280BD133462A46394604A857
:10F7C00004F0B6FA002803D1049870B903E00E20C3
:10F7D00008B0BDE8F0810748009033462A46394614
:10F7E000404600F0B9F90028F2D1019820600020CD
:10F7F000EEE700008D3D02007CB50C46D0B12CB187
:10F8000000230193057801A9652D01D007207CBD57
:10F810000125019572B1156865B1009313460A463A
:10F82000214600F06BF90028F1D10198A04203D0E5
:10F8300009207CBD0E207CBD00207CBD2DE9FF4150
:10F8400084B0984614460F0019D0C4B1002001902E
:10F850002568652001AE8DF8080033462A4602A8C7
:10F8600004F094FA00280BD133462A46394604A8FE
:10F8700004F05EFA002803D1049870B903E00E206A
:10F8800008B0BDE8F0810748009033462A46394663
:10F89000404601F0A1FE0028F2D10198206000202E
:10F8A000EEE70000A9F801002DE9F0411D461746DA
:10F8B0000E0016D0ADB1A0B1044604F067FA0028DE
:10F8C00010D12B463A463146A01C04F000FA00281D
:10F8D00008D12B463A463146201DBDE8F04104F0E0
:10F8E000F6B90E20BDE8F0812DE9F84F4FF0000881
:10F8F000DDE90AA681468DF8008010680F461C4697
:10F900001546B84216D06B46484604F027FA9DF8D3
:10F910000000012805D00CB1C4F800800020BDE82B
:10F92000F88F4CB1206838B1564503D829687A1A47
:10F93000B24203D20920F2E70E20F0E749443246F2
:10F94000F9F77AFC286830442860E7E72DE9F843A6
:10F950009846089C91460D46060001D0012000E023
:10F9600000208DF80000234642464946684604F0D0
:10F970000DFA070006D17EB12068A8EB0001A9426C
:10F9800002D20920BDE8F88348442A463146F9F7F7
:10F9900053FC2068284420603846F3E7184810B527
:10F9A0000178427801F00F01FF2A16D8154B5B7AD7
:10F9B000032B01D0042B01D102290ED831B101292A
:10F9C0000DD002290DD003290DD006E00E49801C70
:10F9D000F9F756FC08B9012010BD002010BD0F2317
:10F9E00002E0552300E0FF23002105E04418A4783D
:10F9F0009C42F2D1491CC9B29142F7D3EBE7000017
:10FA0000D432002050270020043E020070B5084C7C
:10FA1000050009D010342168002907D0086820604B
:10FA2000496828468847F6E70834F4E770BD0000C7
:10FA3000D8330020054A012120B1012805D1917059
:10FA4000FFF7E4BF51700020FAE77047D833002079
:10FA50002DE9F05F26484168F1B3DFF898B00E68F1
:10FA60008146DBF8004087688078E11B21F07F4504
:10FA7000ED1CB0B9DFF880804FF48030C8F8440343
:10FA8000C8F804031120F9F751FC1120F9F759FCCB
:10FA90004FF0010AC8F800A02F2002F055FD89F8A8
:10FAA00002A0B54200D23546124BE8193C3320F093
:10FAB0007F401860DBF800105A46091B21F07F4197
:10FAC000001B20F07F40C91C81420FD910681860CC
:10FAD0002F2002F039FD00E004E0BDE8F05F1120C6
:10FAE000F9F73ABCBDE8F05F03F058B8BDE8F09F05
:10FAF000B827002004150140001001402DE9F8430B
:10FB00008846116881460025089E1C4617464046D7
:10FB1000414502D10920BDE8F88301466B464846BD
:10FB200004F01CF99DF80000012803D078B10B25E2
:10FB30002846F0E74CB123683BB1002EF8D03A4696
:10FB400041464846B0470546F2E70E20E3E7002C61
:10FB5000EED000202060EBE7F0B41C6806460020E1
:10FB6000049D671C974202D90920F0BC7047002E03
:10FB700002D04FF0010701E04FF000070F551C685D
:10FB800004F101041C60F0D0002DEED03046AC46EC
:10FB9000F0BC60471149002202EB821351F8233078
:10FBA000834204D102EB821001EB800014E0521C6E
:10FBB000082AF1D35FF0000202EB821351F82330E0
:10FBC00023B1521C082AF7D30020704702EB82129F
:10FBD00041F8220001EB8200001D7047883E0020A2
:10FBE000034610B504200D4A002100BFC1EB0114EB
:10FBF00004EB840402EB8404A4781CB1491C08299A
:10FC0000F4D310BDC1EB011404EB840402EB8402B5
:10FC1000012090700020196010BD000028350020E0
:10FC2000034610B505200C4A002100BFC1EB0114AA
:10FC300004EB840432F824409C4208D1C1EB01114A
:10FC400001EB810102EB81010020887010BD491C8D
:10FC50000829EBD310BD00002835002070B50446FC
:10FC600005200B4B002200BFC2EB021505EB8505FA
:10FC700033F82560A64204D103EB8505AD78012D4C
:10FC800003D0521C082AEFD370BD00200A6070BD5B
:10FC900028350020034610B504200E4A002100BF7D
:10FCA00001EB410404EB011402EB8404A4781CB1C1
:10FCB000491C0829F4D310BD01EB410000EB0110F1
:10FCC00002EB80000124847000F10C0242600020ED
:10FCD000196010BDA8460020034610B505200C4A47
:10FCE000002100BF01EB410404EB011432F8244071
:10FCF0009C4209D101EB410303EB011102EB8101AD
:10FD000000208870486010BD491C0829EAD310BD46
:10FD1000A846002070B5044605200B4B002200BF0A
:10FD200002EB420505EB021533F82560A64204D12B
:10FD300003EB8505AD78012D03D0521C082AEFD3C3
:10FD400070BD00200A6070BDA846002070B5C6B026
:10FD50001C461546D8B1D5B1CCB10E4A40921646D4
:10FD6000F822ADF80E2141AA3E92CDF808D13EAB63
:10FD70003FAAF9F7A9FE002807D1DDE93E10324677
:10FD800069DF22462946F9F71FFF46B070BD0E20F5
:10FD9000FBE70000502700207CB51C46154680B1CB
:10FDA0007DB174B1084A01920092FAF705F8002873
:10FDB00006D1684602F06CFA22462946FAF70BF89B
:10FDC0007CBD0E207CBD0000502700203EB51C46A7
:10FDD000154688B185B17CB101AA009289B26A4604
:10FDE000FAF753F9002806D100986DDF224629461C
:10FDF000009BFAF769F93EBD0E203EBD3EB51C469C
:10FE0000154678B175B16CB101AA00926A46FAF74D
:10FE10008DF9002805D100986CDF22462946FAF7B3
:10FE2000A7F93EBD0E203EBD30B591B01C4615462B
:10FE300030B32DB324B310AA019204AA0292002277
:10FE4000049206920EAA4FF48073099208AAADF8A4
:10FE50001430039203AAADF81C30009289B202ABB1
:10FE600001AAFAF787FA002808D101AB93E8070046
:10FE700072DF22462946019BFAF7C6FA11B030BD5F
:10FE80000E20FBE77CB51C46154688B185B17CB1D8
:10FE90006B4601AAFAF7EEFA002808D19DF8001087
:10FEA0009DF8040073DF22462946FAF70BFB7CBD60
:10FEB0000E207CBD38B51C46154678B175B16CB1C5
:10FEC00089B26A46FAF704FB002806D19DF80000C3
:10FED00074DF22462946FAF719FB38BD0E2038BDDB
:10FEE0007CB51C46154688B185B17CB101AA00924B
:10FEF00089B26A46FAF710FB002806D1009879DF2C
:10FF000022462946009BFAF729FB7CBD0E207CBDCA
:10FF100038B51C46154670B16DB164B16A46FAF742
:10FF200053FB002806D1BDF8000078DF22462946A1
:10FF3000FAF769FB38BD0E2038BD30B589B01C46D4
:10FF40001546C0B1BDB1B4B104AA019201AA009294
:10FF500089B203AB02AAFAF75CFB002809D19DF82D
:10FF60000C10BDF80800019A80DF22462946FAF7F6
:10FF700093FB09B030BD0E20FBE77FB51C4615464C
:10FF800098B195B18CB102AA00926B4601AAFAF71A
:10FF900089FB002807D1BDF8040000997EDF2246C6
:10FFA0002946FAF7B1FB04B070BD0E20FBE77FB520
:10FFB0001C46154698B195B18CB102AA00926B46C9
:10FFC00001AAFAF71BFC002807D1BDF8040000992C
:10FFD00075DF22462946FAF743FC04B070BD0E20B7
:10FFE000FBE73EB51C46154698B195B18CB102AA07
:10FFF00000926B4601AAFAF789FC002808D1BDF8E7
:020000040002F8
:100000000400009987DF23462A460099FAF7AAFCE4
:100010003EBD0E203EBD0000F0B5E3B01C461546C7
:100020008E4660B35DB354B3002201AE4FAB2FAF29
:100030000DF5B471C2EBC20C0CEB021CB44443F8D6
:1000400022C007EB021C41F822C0521CD2B2082A7F
:10005000F0D3CDE9573159A9009158AB57AA714651
:10006000FAF7F8FC002808D1DDE957019DF8642172
:100070006FDF22462946FAF76BFD63B0F0BD0E2014
:10008000FBE730B5C3B01C461546B0B1ADB1A4B165
:1000900001AA3F9241AA409240AB3FAAFAF75EFD07
:1000A000002808D1DDE93F017DDF0094DDE93F1242
:1000B0002B46FAF783FD43B030BD0E20FBE730B589
:1000C000C3B01C461546D8B1D5B1CCB142AA3F92B7
:1000D00001AA4092F822ADF8042141AA009240AB57
:1000E0003FAAFAF7ADFD002808D1BDF80421DDE9EB
:1000F0003F017CDF22462946FAF7D8FD43B030BDE8
:100100000E20FBE77CB51C46154688B185B17CB155
:1001100001AB6A46FAF7D0FD002808D19DF804101B
:10012000BDF8000076DF22462946FAF7EFFD7CBDD8
:100130000E207CBD7CB51C46154688B185B17CB1CE
:1001400001AB6A46FBF700FC002808D19DF80410BB
:10015000BDF8000082DF22462946FBF71FFC7CBD6C
:100160000E207CBD30B58BB01C46154698B195B1BC
:100170008CB102AA00926B4601AAFBF715FC00287D
:1001800007D1BDF80400009981DF22462946FBF71C
:100190003BFC0BB030BD0E20FBE730B59FB01C46DA
:1001A0001546C8B1C5B1BCB114AA019203AA029206
:1001B00001AA009202AB13AAFBF738FC002809D170
:1001C000DDE90121BDF84C0083DF23462A46019971
:1001D000FBF76CFC1FB030BD0E20FBE730B599B0CB
:1001E0001C461546C0B1BDB1B4B104AA01920EAA15
:1001F000029202AA009201AB03AAFBF78DFC002831
:1002000008D1DDE90112BDF80C0084DF2246294641
:10021000FBF7C2FC19B030BD0E20FBE73EB51C4613
:10022000154690B18DB184B102AA00926B4601AA25
:10023000FBF722FE002807D1BDF8040000998FDFEC
:1002400022462946FBF74AFE3EBD0E203EBD3EB586
:100250001C46154688B185B17CB101AA009289B2CD
:100260006A46FBF771FE002806D100987BDF224624
:100270002946009BFBF78CFE3EBD0E203EBD3EB5E1
:100280001C46154678B175B16CB101AA00926A4658
:10029000FBF7B4FE002805D100987ADF22462946F4
:1002A000FBF7D0FE3EBD0E203EBD30B587B01C46EC
:1002B0001546A0B19DB194B101AA009203AA029281
:1002C00089B26A46FBF7C4FE002806D1009871DFA8
:1002D00022462946009BFBF7DDFE07B030BD0E200D
:1002E000FBE730B587B01C46154690B18DB184B19F
:1002F00001AA009203AA02926A46FBF755FF002862
:1003000005D1009870DF22462946FBF76FFF07B042
:1003100030BD0E20FBE730B587B01C461546E0B176
:10032000DDB1D4B103AA019205AA029202AA0092F9
:1003300089B201AB04AAFBF75FFF00280BD1DDE90E
:100340000112BDF810008EDF029900912246294665
:10035000019BFBF793FF07B030BD0E20FBE77FB595
:100360001C461546B0B1ADB1A4B103AA009202ABD0
:1003700001AAFBF7C5FF00280AD19DF80C209DF8C3
:100380000810BDF8040088DF22462946FBF7F1FF7C
:1003900004B070BD0E20FBE738B51C46154670B1A1
:1003A0006DB164B16A46FBF7EAFF002806D1BDF8DB
:1003B000000089DF22462946FCF700F838BD0E20F0
:1003C00038BD30B595B01C461546F0B1EDB1E4B17D
:1003D00008AA02920DAA039211AA049204AB03AADE
:1003E000CDE9002389B202AB07AAFBF7EDFF002895
:1003F00009D102A890E80E00BDF81C0086DF224655
:100400002946FCF737F815B030BD0E20FBE7000099
:100410002DE9F04188B01D461646884607003DD0BC
:10042000DEB3D5B30020059006A8039005A8FFF71A
:10043000D7FB002833D105982349C0EB001000EB0F
:10044000800001EB8004201D04F124020290626010
:10045000059A04ABC2EB021202EB820201EB8201AD
:1004600001F14002A2601732E26010322261413293
:1004700062611C3242611732EB31C0E9062102A9E8
:1004800003A8CDE90001224641463846FCF7FCF8B6
:10049000002804D1029828B109E0FFE70E2008B037
:1004A000BDE8F0812088FFF7BBFB0028F7D1DDE92C
:1004B000023220889DF810107FDF2A463146029BC9
:1004C000FCF732F9EBE70000283500207FB51C4629
:1004D0001546B0B1ADB1A4B101AA009203AB02AA16
:1004E000FCF71EFA00280AD19DF90420BDF80C1073
:1004F0009DF8080077DF22462946FCF745FA04B04C
:1005000070BD0E20FBE70000F0B599B01C46154603
:100510000E4600B3FDB1F4B100226B460DF1380177
:10052000C2EBC2071F4441F82270521CD2B2082A03
:10053000F6D3169117AB16AA3146FCF72BFA002812
:1005400007D19DF85C1016986EDF22462946FCF70D
:100550006FFA19B0F0BD0E20FBE73EB51C461546FC
:10056000A8B1A5B19CB10023029302AB009301AAEC
:1005700089B26B46FCF714FB002807D1BDF80400D4
:1005800000999FDF22462946FCF73CFB3EBD0E202A
:100590003EBD30B587B01C461546D8B1D5B1CCB1FB
:1005A0000022049204AA019205AA029202AA0092D1
:1005B00089B201AB03AAFCF76BFB002808D1DDE987
:1005C0000112BDF80C00A0DF22462946FCF7A4FB6F
:1005D00007B030BD0E20FBE730B58BB01C4615468A
:1005E000D8B1D5B1CCB104AB01930B23ADF8083031
:1005F00002AB009303AA89B201ABFCF793FB00287E
:1006000009D1BDF80820BDF80C000199A2DF2246EF
:100610002946FCF7B9FB0BB030BD0E20FBE73EB519
:100620001C46154698B195B18CB102AA009289B2C8
:100630006B4601AAFCF7AEFB002807D1BDF8040009
:1006400000999DDF22462946FCF7D2FB3EBD0E20D5
:100650003EBD3EB51C46154698B195B18CB102AA77
:10066000009289B26B4601AAFCF7EAFB002807D189
:10067000BDF8040000999EDF22462946FCF70EFCD7
:100680003EBD0E203EBD7CB51C46154690B18DB1D9
:1006900084B189B201AB6A46FDF763F9002808D13D
:1006A000BDF80410BDF80000A5DF22462946FDF77D
:1006B00080F97CBD0E207CBD7CB51C46154688B1FA
:1006C00085B17CB16A4601ABFDF7A9F9002808D1D4
:1006D000BDF80410BDF80000A4DF22462946FDF74E
:1006E000C6F97CBD0E207CBD30B585B01C461546D4
:1006F000C0B1BDB1B4B104AA019201AA009289B2FD
:1007000003AB02AAFDF7D4F9002809D1BDF80C10FB
:10071000BDF80800019A9BDF22462946FDF700FA42
:1007200005B030BD0E20FBE77FB51C461546B8B1BD
:10073000B5B1ACB103AE01AA02AB89B20096FDF728
:10074000F5F900280AD1BDF80C20BDF80810BDF855
:100750000400A1DF22462946FDF71CFA04B070BD53
:100760000E20FBE73EB51C46154698B195B18CB1FD
:1007700002AA009289B26B4601AAFDF711FA00287D
:1007800007D1BDF8040000999CDF22462946FDF7F9
:1007900035FA3EBD0E203EBD30B5C3B01C461546F1
:1007A000E0B1DDB1D4B100233F9340933FAB3D9323
:1007B000F423ADF802313EAACDF804D189B23DABA5
:1007C000FDF770FA002807D1BDF8F8003D99A3DFC6
:1007D00022462946FDF794FA43B030BD0E20FBE7D0
:1007E00030B587B01C461546D8B1D5B1CCB104AAF6
:1007F000019205AA029201AA009202AB03AAFDF798
:1008000085FA00280BD1DDE90121BDF80C00B4DF29
:100810000199009122462946029BFDF7ADFA07B0E7
:1008200030BD0E20FBE770B5ADF58E6D1C4615464C
:100830000E46F0B3EDB3E4B302AACDF830240DF5C3
:100840008962CDF838241032CDF83C24121DCDF841
:100850004024121D4FF40071CDF84424ADF8361435
:10086000343ACDF80C24ADF82014383282A9CDF8F2
:100870001824CDF82814121D0DF58361CDF81C2421
:10088000CDF810143831CDF808144039603ACDE96C
:1008900000120B1F0A1D3146FDF76AFC00280FD11C
:1008A0000DF20C41BDF8140406C9DDF80834AADFC6
:1008B00000E008E022462946DDF80834FDF79EFCFA
:1008C0000DF58E6D70BD0E20FAE730B5ADF50D7DDE
:1008D0001C46154620B31DB314B384AA829289AA7C
:1008E00084928AAA859201AA88924FF40072ADF888
:1008F00018228BAA819281AA009282AB83AAFDF76B
:10090000BBFC002809D1DDE98121BDF80C02ABDF79
:1009100022462946819BFDF7E9FC0DF50D7D30BD92
:100920000E20FAE77CB51C46154690B18DB184B116
:100930006A4601AB89B2FDF7AFFF002808D1BDF8C8
:100940000410BDF80000B5DF22462946FDF7CCFFB4
:100950007CBD0E207CBD70B5ADF5087D1C461546EE
:100960000E46D0B1CDB1C4B14FF4007282ABADF838
:1009700018228093694686AACDE9842180AB81AA9A
:100980003146FDF7F3FF002808D1BDF80402809935
:10099000AEDF809929B18B6804E00E200DF5087D4B
:1009A00070BD002322462946FEF70EF8F6E730B563
:1009B00085B01C461546C8B1C5B1BCB104AA0192A8
:1009C00001AA009289B203AB02AAFEF733F800280D
:1009D0000AD1BDF80C10BDF80800019AA9DF224623
:1009E0002946019BFEF75CF805B030BD0E20FBE701
:1009F0007CB51C46154680B17DB174B101AA009248
:100A00006A46FEF783F8002806D10098B3DF224635
:100A10002946009BFEF79AF87CBD0E207CBD30B5C0
:100A2000ADF5077D1C461546D0B1CDB1C4B182AA43
:100A300080924FF40072ADF81222CDF814D280AB40
:100A400081AAFEF7D9F8002807D1BDF804028099E1
:100A5000B0DF22462946FEF7FDF80DF5077D30BDD3
:100A60000E20FAE730B587B01C461546D8B1D5B18F
:100A7000CCB10022049204AA029205AA019201AA12
:100A8000009202AB03AAFEF7EBF8002809D1DDE9DA
:100A900001219DF80C00A8DF22462946019BFEF7A4
:100AA00019F907B030BD0E20FBE77FB51C4615468F
:100AB000B0B1ADB1A4B103AA009202AB01AAFEF796
:100AC0003FF900280AD1BDF80C20BDF80810BDF888
:100AD0000400AFDF22462946FEF766F904B070BD78
:100AE0000E20FBE730B5ADF5077D1C46154618B363
:100AF00015B30CB302AA82924FF40072ADF818221B
:100B000086AA839285AB83AACDE9002382AB84AA0F
:100B1000FEF750F900280CD1DDE98212BDF8100271
:100B2000859BB2DF8399009122462946829BFEF77E
:100B300083F90DF5077D30BD0E20FAE730B5ADF530
:100B4000077D1C461546F8B1F5B1ECB102AA8292B8
:100B50004FF40072ADF80C2285AB83AACDE90023D7
:100B600082AB84AAFEF7AAF900280AD1BDF80C22AC
:100B7000BDF81002859B8299B1DF22462946FEF717
:100B8000D2F90DF5077D30BD0E20FAE730B5ADF591
:100B9000077D1C461546E0B1DDB1D4B184AA81922F
:100BA00001AA859281AA009289B283AB82AAFEF73C
:100BB000C0F900280AD1BDF80C12BDF80802819ACC
:100BC000ADDF22462946819BFEF704FA0DF5077D2D
:100BD00030BD0E20FAE7000030B5ADF5077D1C46AC
:100BE0001546F8B1F5B1ECB10F4A89B283AB126882
:100BF000849201AA859284AA819281AA009282AAF3
:100C0000FEF71EFA00280AD1BDF80C12BDF8080242
:100C1000819AACDF22462946819BFEF749FA0DF501
:100C2000077D30BD0E20FAE73841020030B589B0AB
:100C30001C46154680B17DB174B102AA019289B2F9
:100C400001AB04AAFEF798FA002806D104982128DF
:100C500005D0222808D105E00E2009B030BD07A933
:100C6000039101E005A90291019968DF01990091C2
:100C700022462946049BFEF7AFFAEEE7F0B587B0AF
:100C80001D4616460C46070013D096B18DB14FF0A5
:100C9000FF300090A1B26A463846FEF703FB0028F9
:100CA00008D102A801900098212805D0222808D157
:100CB00005E00E2007B0F0BD06A8039001E004A8EF
:100CC0000290A1B201AB6A463846FEF701FB00284C
:100CD000F0D1DDE9000167DF2A463146FEF766FB09
:100CE000E8E7000030B585B01C46154658B355B34B
:100CF0004CB303AA019201AB6A46FEF7A9FB002898
:100D00001FD10198A8B102A8FEF7C4FF002818D18E
:100D10000298BDF8002000EB400101EB00110B48E8
:100D200020F82120019A00EB810092880281001DA9
:100D300001900146BDF8000066DF22462946FEF715
:100D4000B9FB05B030BD0E20FBE70000A84600202F
:100D500030B589B01C461546E0B1DDB1D4B11022E2
:100D60008DF8082004AA039208AA019201AA009211
:100D700003AB02AAFEF7BCFB002809D19DF80800CE
:100D8000019A039963DF22462946019BFEF7DCFBAB
:100D900009B030BD0E20FBE730B58BB01C461546C0
:100DA00018B315B30CB310228DF8102004AA0292C8
:100DB00005AA019209AA03920022099201AA0092AF
:100DC00089B202AB03AAFEF7F5FB00280BD1DDE9DF
:100DD0000210019A64DF019900919DF810302246BB
:100DE0002946FEF72FFC0BB030BD0E20FBE730B5D7
:100DF00087B01C461546B0B1ADB1A4B102AA0192AC
:100E000006AA009289B26B4601AAFEF789FC002867
:100E100007D1DDE9001062DF22462946009BFEF77C
:100E2000B5FC07B030BD0E20FBE73EB51C461546AD
:100E300088B185B17CB101AA009289B26A46FEF7F9
:100E4000DBFC002806D1009865DF22462946009B7E
:100E5000FEF7F4FC3EBD0E203EBD30B58DB01C4605
:100E6000154688B185B17CB1CDF830D00CAA00F020
:100E700009FB002806D10C9846DF224629460C9B28
:100E800000F022FB0DB030BD0E20FBE7F0B480B1C6
:100E90007AB173B105780B4E002400BF16F8347098
:100EA000AF4209D106EBC404646844B1A446F0BC67
:100EB00060470E20F0BC7047641C452CEED3062022
:100EC000F8E70000103F020010B540B13AB133B16D
:100ED00089B201F09FFD002800D133DF10BD0E2044
:100EE00010BD7CB51C46154680B17DB174B101AA18
:100EF00000926A4602F0A8FB002806D100984CDF59
:100F000022462946009B02F0BFFB7CBD0E207CBD23
:100F10002DE9FC430024099E1D461746884681465C
:100F2000ADF800408DF8044056B14DB1286838B195
:100F30003968A8EB0100032804D20920BDE8FC832E
:100F40000E20FBE76B464146484602F0A5FE30887E
:100F5000BDF80010884201D20C20EFE701AB3A4601
:100F60004146484602F0FAFE9DF8040008B100240C
:100F70000EE0BDF8000030802C600EE028683A4694
:100F800000EB44034146484602F086FE641CA4B2CE
:100F9000BDF800008442F1D334800020CEE710B5C4
:100FA000044612B11088002211E04FF6FF70FAE7F4
:100FB000030A43EA0023A05C5840C0F303135840DF
:100FC00080EA003080B2C3B280EA4310521C8A42E9
:100FD000EED310BD2DE9F05F884C0E46174614F88D
:100FE000381F02F03F0201F0C00111434AC414F857
:100FF0003B2C443C032A01D0042A03D1032B01D10A
:10100000FF22E2630125A5724FF00008A4F80E80CC
:10101000227862B14FF0030A4FF0040948B1032867
:101020004AD0012A51D0E5810220BDE8F09F052079
:10103000FBE700F0C3F956B1012E11D0022E14D0F7
:10104000032E23D0042E24D0052E25D0A9E0002F76
:1010500055D1C4F8388084F809A084F80580A7E049
:10106000032F4CD8B801A063A2E0012F02D0022FB9
:1010700045D104E084F809A084F8058002E084F8F2
:1010800009906571BDE8F05F01F0E0BC012F36D832
:101090008EE0A7BB06200BE04FF4FF7047B144F28F
:1010A0009021012F06D0022F02D0032F79D101E029
:1010B000E0817DE0E1817BE0012AB4D0A08940F4A9
:1010C0000040E08100F07AF972E0032B04D0272E73
:1010D00002D9E5810120A8E74246A4F80C80012846
:1010E00002D002280CD063E040F201114448F8F726
:1010F000BCF8012001F004FD84F8009058E050E0B5
:10110000E36BFF2B04D0FF2902D9E58103208CE794
:101110003B48DFF8F0B04FF002084170022B14D0CA
:1011200003DC3BB1012B3CD10BE0032B1DD0FF2B8B
:1011300037D11EE000F8022B0A463349F8F77CF855
:1011400008E000F8025B0F2202E000F8028B552253
:10115000F8F784F8002001F0D3FC627A0020A16B3C
:10116000042A27D0032A27D027E000F8029BFF2279
:10117000EEE7304637B1012F04D0022F0ED0032FF7
:1011800016D111E0002001F0BBFC00F041F8CBF8D3
:101190000052CBF8005084F800A009E000F0AAF853
:1011A00004E0E581042040E700F094F80028F8D03E
:1011B00000203AE7582000E0502000EBC101042A4B
:1011C00000D149080020F93140F27122401C42430D
:1011D0009142F9D840F271214843A169C1F8400514
:1011E0000A4801F5A0710160011DC1F800B007486F
:1011F0000C38056084F80080DAE7000050270020F2
:10120000D432002000100040043E020010F50140DE
:1012100002494FF40070086070470000501600400B
:10122000034900238A7A8B72C9890160104670478E
:10123000502700202AB1012A07D0022A09D0002015
:101240007047074A0260082006E0064A026009204B
:1012500002E0054A02600A20087001207047000081
:10126000008000400090004000A0004010B502F057
:1012700041FA10B901F0EAFB08B1042010BD06489C
:10128000002101228172027081630448016841F0EB
:1012900010010160002010BD5027002010ED00E07B
:1012A00078B104280DD0D8280BD0EC2809D0F0282C
:1012B00007D0F42805D0F82803D0FC2801D0032853
:1012C00003D1032903D0042901D004207047002052
:1012D0007047000006490978012901D900207047AC
:1012E00003490246491C01F11700FFF7A3BF0000A4
:1012F0005027002040B210F0300F01D040F0C00065
:10130000044940B20A78012A01D900207047486197
:101310000120704750270020F3B5002683B03746E0
:10132000344603A802F0F0FB00280DD1FFF79EFF22
:1013300048B900BF00F05AF805461F486946012227
:1013400001F04CF910B1032005B0F0BD5FB11A48AF
:10135000603800683044A84207D200BF9DF8000002
:101360002E460402E6E70127F8E79DF80000002773
:101370000443A00BC4F30521C4F3850204F0030366
:10138000FFF728FE02A8FFF74BFF0028D2D00298F3
:101390000122000A8DF80400074801A9001F00F08F
:1013A00036FE02988DF804000348012201A9001FAF
:1013B00000F02DFEBEE700002C28002010B500F044
:1013C00013F807480124046005490020083108602B
:1013D000091D086001F0C4FB0248047010BD000044
:1013E00008F5014050270020704700002DE9F04724
:1013F0001F48016841F0100101601E4D0127DFF810
:1014000078801E4C40F20119002600BFD5F80C016F
:10141000B0B1C5F80C610120F7F77DFF20780428F2
:101420000ED16F60D8F80000012805D1FEF7B6FA9A
:1014300010B1A089401CA08149461148F7F715FF5B
:10144000A069D0F8401111B1C0F84061DEE7D0F8D2
:1014500044010028DAD0A069C0F8446194F9010081
:10146000F7F759FF2069401C2061BDE8F0870000B4
:1014700010ED00E000100040001400405027002054
:10148000D43200201CB50C4640B12CB10021019192
:10149000037801A9462B03D007201CBD0E201CBDDC
:1014A00001230193074B009313460A462146FEF79A
:1014B00025FB0028F3D10198A04201D009201CBDD2
:1014C00000201CBD1B2002002DE9FF4184B098467E
:1014D00014460F0019D0C4B10020019025684620A1
:1014E00001AE8DF8080033462A4602A802F04EFCF1
:1014F00000280BD133462A46394604A802F018FCCE
:10150000002803D1049870B903E00E2008B0BDE8AC
:10151000F0810748009033462A4639464046FEF798
:101520001BFB0028F2D1019820600020EEE70000AC
:10153000532002000E4910B50A784C780023A242CD
:1015400012D0521CD2B20A70022A00D10B70084A83
:101550000B780C3252F8232002608868104420F087
:101560007F408860012010BD0360002010BD000096
:10157000B8270020034890F82800401C00F007001E
:10158000704700005428002030B4029C1CB113B1F5
:10159000A44630BC604730BC0E20704730B4029C7B
:1015A0001CB113B1A44630BC604730BC0E2070475C
:1015B00030B4029C1CB113B1A44630BC604730BCAF
:1015C0000E20704730B4029C1CB113B1A44630BC4D
:1015D000604730BC0E20704730B4029C1CB110B183
:1015E000A44630BC604730BC0E20704730B4029C2B
:1015F0001CB110B1A44630BC604730BC0E2070470F
:1016000030B4029C1CB110B1A44630BC604730BC61
:101610000E20704730B4029C1CB110B1A44630BCFF
:10162000604730BC0E20704730B4029C1CB110B132
:10163000A44630BC604730BC0E20704730B4029CDA
:101640001CB110B1A44630BC604730BC0E207047BE
:1016500030B4029C1CB110B1A44630BC604730BC11
:101660000E20704730B4029C1CB110B1A44630BCAF
:10167000604730BC0E20704730B5234D87B005F170
:101680001C0495F8280095F8241040EAC10040F0A9
:10169000C000207035F80C0F0E2141EA0010607078
:1016A000000AA070204600F0ABFAE070002204218E
:1016B0002046FFF774FCADF800006A462988A86848
:1016C000FFF76DFCA4F11401ADF800000870000AEA
:1016D000487004200194ADF80800A8680390288899
:1016E000ADF81000084605900220ADF8180005AAD4
:1016F00003A901A801F030FE002802D00020F8F76D
:1017000083F807B030BD000054280020064890F848
:101710002810491C002301F007014361816263F333
:10172000070001F0B1BD00005428002010B580680A
:1017300001F0F4FD002804D0BDE810400020F8F7C7
:1017400063B810BD38B5054600248DF800406846E2
:10175000F8F738F929460D4800F01DFD10B10020BA
:10176000F8F752F80A48C178C279114208D0C4701B
:101770009DF80000F8F74AF9BDE8384000F00AB8D3
:101780009DF80000F8F742F938BD000064420200FD
:101790005428002010B586B05FF000048DF810408A
:1017A00004A8F8F70FF9002269460A4800F08DFCFA
:1017B00040B109490120C8709DF81000F8F726F9DA
:1017C00006B010BD9DF81000F8F720F9684600F04B
:1017D00005F8E3E764420200542800202DE9F041B7
:1017E0003F4C0346204694F801C002260125016BB8
:1017F000BCF1010F10D0428903270069BCF1020F30
:1018000032D0BCF1030F48D0BCF1040F5CD0BDE86E
:10181000F0410020F7F7F8BF187801281CD118799B
:10182000022819D19A6894F82470107800F0070003
:10183000874213D12571226398896081062802D8D6
:101840000020F7F7E1FF638965F307009B1F63F34F
:101850000F0101F019FD6670BDE8F0810420607091
:10186000084601F05BFD14E01D78002DF4D11B79D2
:10187000012BF1D130B1091D921FF7F7DDFC206B70
:1018800001F04CFD677094F82400401C00F0070044
:101890006062BDE8F041F7F773BF19780129DBD129
:1018A0001979012902D0022914D0D5E730B10146B7
:1018B000931F66F3070063F30F0201E067F307006D
:1018C00001F0E2FC6570C7E71878012802D11879A9
:1018D0000128F7D09868BDE8F04101F01FBD000075
:1018E000542800201FB502208DF8000000208DF83C
:1018F0000400684600F0BEF81FBD00007FB5027806
:1019000001217AB1012A13D0022A3ED18DF80010AC
:1019100001788DF80410416802910089ADF80C003F
:1019200079B90BE08DF8001000788DF8040029E0FB
:101930008DF8001000788DF8040043E00020F7F7E0
:1019400063FFBDF80C0010B90020F7F75DFFBDF88C
:101950000C500298042D39D3407800F00F02052A6C
:1019600003D07AB10E2A11D030E0BFF34F8F1C485C
:1019700001681C4A01F4E06111430160BFF34F8F1D
:1019800000BFFDE7684600F075F87FBD029C042D9E
:101990001CD921784B0619D50B0617D50E2A15D15F
:1019A0000844A178E2781144084410F0FF0F0DD1EB
:1019B00000222046A91EFFF7F2FA611931F8021C35
:1019C000884203D16846FFF7BDFE7FBD029801F053
:1019D000A5FC0028F9D00020F7F716FF7FBD000016
:1019E0000CED00E00400FA0530B50D494FF400326B
:1019F0000124C1F8082388B1FA235843094BC0EBEE
:101A000040151D601D6805EB90001860CC6000203B
:101A1000C1F844010C60C1F8042330BD4C6030BDF6
:101A200000A0004044A500400F4910B509200860FF
:101A30000D4900200C390860091D08600B4901227E
:101A4000CA60421EC1F808234FF40032C1F80423D3
:101A50004FF0E0220915C2F88012054C402384F8AB
:101A60000034C2F8001110BD10A5004000A00040D5
:101A70000AE000E038B5054600248DF800406846CD
:101A8000F7F7A0FF29460D4800F085FB10B10020B4
:101A9000F7F7BAFE0A488178C279114208D08470FB
:101AA0009DF80000F7F7B2FFBDE8384000F00AB833
:101AB0009DF80000F7F7AAFF38BD00005042020071
:101AC0005428002010B586B05FF000048DF8104057
:101AD00004A8F7F777FF002269460A4800F0F5FAF4
:101AE00040B10949012088709DF81000F7F78EFF7A
:101AF00006B010BD9DF81000F7F788FF684600F0AB
:101B000005F8E3E750420200542800202DE9F04197
:101B10003A4D04460427287801264FF00508062888
:101B200067D2DFE800F066031523355C207818B132
:101B3000012816D1207916E02079002811D1FFF76D
:101B40009BFD0020FFF750FF0220C5F82C802BE002
:101B50002078012805D1207928B90120FFF744FF1A
:101B60002F70BDE8F08102282DD0FAE720780128F7
:101B7000F7D120790028F0D00228F2D1A06801F036
:101B80002BF800B30020FFF72FFF85F800801AE044
:101B9000207801280AD00228E3D1E86A401EE862D2
:101BA00016D0FFF769FD03202870DAE720790228B4
:101BB000D7D1A06801F010F828B10020FFF714FF7A
:101BC000FFF7A4FD2E702046BDE8F041FFF7AEBD43
:101BD000062262F307006A6901F056FB07E02078ED
:101BE0000128BED120790028BDD1FFF78FFD2E70CE
:101BF000B7E7BDE8F0410020F7F706BE5428002003
:101C000001784278807811440844C043401CC0B237
:101C10007047000070B50D46044600684FF48871A7
:101C200000F04CFC4FF49071206800F047FC4FF43A
:101C30009271206800F042FC4FF4A271206800F01D
:101C40003DFC20681249C0F8041320686907000BA6
:101C500040B2090E002806DA00F00F0000F1E02083
:101C600080F8141D03E000F1E02080F800142068E3
:101C70000121000B40B200F01F029140400980009A
:101C800000F1E020C0F88012C0F8001170BD000023
:101C9000100302000268134602E08A4204D0126870
:101CA000002AFAD10B60016070472DE9FC471E46FF
:101CB0000A9C1746884681462588234601F0F8FF8E
:101CC000002808D120883346CDE900503A464146E5
:101CD0004846FDF709FEBDE8FC87FFB581B01D460B
:101CE00016460A9C074623462A46314602A801F0BA
:101CF000EEFF002807D12B4632460094BDF80810AD
:101D00003846FDF723FE05B0F0BD2DE9FC471E4621
:101D10000A9C1746884681462578234602F029F812
:101D2000002808D120783346CDE900503A46414694
:101D30004846FDF7D9FDBDE8FC8700002DE9F047D6
:101D4000394E002780463D46DFF8E090D6F804A0E3
:101D500057E003D00446D0F81C8035E099F8002005
:101D600002EB4201521CD2B289F8002009EBC101FA
:101D700099F80230091D9A4201D189F8005048684B
:101D80000A780446012A12D0022A02D0032A3BD143
:101D900008E001F03DFD00B10127257434E0057431
:101DA000C06900E070680028F9D170602CE0207CE8
:101DB00050BB88686060C868A0600869E0604869D6
:101DC000A061F07800B165606268B168184B501A84
:101DD00020F07F40984202D2A168084406E0881AA9
:101DE000A16820F07F40814202D9081A206000E0FB
:101DF000256065600120A56020742046E56101F042
:101E0000E9FCB8F10000A4D199F8001099F801009C
:101E10008142A3D117B97168514502D00120BDE8B4
:101E2000F0870020FBE70000B827002010340020D6
:101E3000FFFF7F000120810788671C4A04214FF4BF
:101E4000FE70F7F76DFD08B1F7F7DEFC00F088F8DB
:101E500018B1852801D0F7F7D7FC002000F052F820
:101E600000F03AF80028FBD0114801F0D9F808B189
:101E7000F7F7CAFC00F046FA08B1F7F7C5FC0D48C1
:101E800001F074F8F7F72AFD00F09CFA28B1F7F793
:101E900073FD022801D900F09FFA01F0A5F808B1FE
:101EA000F7F7B2FC00F0CAFCECE70000C028002005
:101EB000E92E02003D28020000F180400068002861
:101EC00000D00120704708B500F18040002101607A
:101ED0000068009008BD000008B500F06DFA30B150
:101EE000684644DF0098002800D0012008BD04485F
:101EF000006800F00110B0F1011FF6D0002008BD0D
:101F00000C040040F8B5154D04466878002648B129
:101F100014B16168002088478DF800606846F7F7C3
:101F200051FD13E08DF800606846F7F74BFD24B1D2
:101F30000A4821460830FFF7ADFE686830B900F066
:101F40003BFA08B142DF01E000F0D4FA6868401CB7
:101F500068609DF80000F7F759FDF8BDD833002000
:101F600070B50B4C207808B185250FE00020A060EB
:101F700060602061E060074800F0C8FA054600F0A4
:101F80001BFA08B900F0A0FA01202070284670BDA5
:101F9000D833002035FA010038B500258DF80050FF
:101FA0006846F7F70FFD074CE068401EE060E06808
:101FB00010B900F0BBFAA5709DF80000F7F726FDF8
:101FC00038BD0000D833002070B5064604780C48B0
:101FD00088B0154640F82420094A0869121D42F8C5
:101FE000240020226846F7F727F904940DB1054A2A
:101FF00000E000226946301D00F0BAFA08B070BD5A
:1020000094270020753B0200001D00F0E7BA001D78
:1020100000F066BB001D00F063BB2DE9F8431646D7
:102020005FEA000813D096B18BB110271C460D460D
:10203000009701F0B8FE002807D104F110033246E2
:1020400029464046009701F0AEFEBDE8F8830E2019
:10205000FBE708B549B143B138B1009313460A46CE
:102060001021203001F0B5FE08BD0E2008BD70B56E
:1020700041EA4201DDE904564FF0A04441EA830100
:1020800041EA052104EB800041EA0641C0F800174F
:1020900070BD1CB5002100910B4601220191FFF794
:1020A000E6FF1CBD1CB500220B46009211460192B2
:1020B000FFF7DDFF1CBD1CB5002100910B4601227E
:1020C00001911146FFF7D3FF1CBD2DE9F8430446EB
:1020D000002790460E468DF800706846F7F772FCB0
:1020E000204600F039F838B105279DF80000F7F7D1
:1020F0008DFC3846BDE8F88320680568B8F1000F0C
:1021000005D10168204600F03FF821680860E268C8
:10211000012A0CD0022A0ED0042A11D06068082AA5
:1021200013D005FB02013046F7F786F8DDE760685B
:10213000405D3070D9E7606830F815003080D4E732
:10214000606850F825003060CFE700EBC501D1E9A9
:102150000001C6E90001C8E70168086849688842CB
:1021600001D1012070470020704701680A68496862
:102170008068884201D9491C00E00021914201D1C8
:1021800001207047002070478068884201D9481CB0
:102190007047002070472DE9F84304464FF00008CF
:1021A0000E468DF800806846F7F70CFC2046FFF7D6
:1021B000DCFF07000AD0207C40B14FF004089DF8F6
:1021C0000000F7F723FC4046BDE8F8832068456827
:1021D00041682046FFF7D8FF2168486037B1206882
:1021E00001682046FFF7D0FF21680860E268012AF5
:1021F00014D0022A16D0042A19D0082A1CD06068EC
:10220000314605FB0200F7F717F8204600F011FCF5
:1022100021688A688242D2D28860D0E761683078CB
:102220004855F2E76168308821F81500EDE76168EC
:10223000306841F82500E8E7D6E90001626802EB62
:10224000C502C2E90001E0E738B5054600248DF873
:1022500000406846F7F7B6FB286804604460846075
:102260009DF80000F7F7D2FB38BD38B504460020D2
:102270008DF800006846F7F7A5FB204600F0D9FB73
:1022800004469DF80000F7F7C1FB204638BD00006A
:1022900060DF002802D1024A01211170704700005E
:1022A000BB28002030B51548ADF5037D0078002827
:1022B00021D04FF4FE7500BFADF8085282A96846E0
:1022C00061DF38B1052816D00DF5037DBDE830403B
:1022D000F7F79ABA6C460A497FA800F0C3F806E0FF
:1022E000D0E90021204690477FA800F0D2F88198DD
:1022F0000028E1D0F4E70DF5037D30BDBB280020B8
:10230000084202007CB5204C207808B108207CBD32
:102310000120A070002000F0D1FC112819D000206D
:1023200000F0E4FC19480026006801908DF8006078
:102330006846F7F747FB164901A810DF05000AD0E9
:10234000002020709DF80000F7F760FB2DB12846B3
:102350007CBD00207CBD0120F3E7A67066700721DC
:10236000162000F061FC08B1F7F74EFA072115209E
:1023700000F05AFC08B1F7F747FA01F03DF90120E7
:1023800000F0B4FCE5E70000B82800209C41020002
:10239000C19701000EB50749684600F063F805E0F3
:1023A000D0E900108847684600F073F802980028CA
:1023B000F6D10EBDB8410200014800787047000018
:1023C000B8280020034801784078814381F001005B
:1023D00070470000B828002070B50C4C6078217858
:1023E000084212D01620F7F7ADF9002530B14FF0B2
:1023F000E0214FF48000C1F8000203E042F2010046
:10240000F7F702FA01F0F8F8657070BDB8280020FF
:102410001FB568464BDF30B1052814D004B0BDE8C5
:102420001040F7F7F1B9084901A800F01BF806E0E1
:10243000D0E900210098904701A800F02AF80398FD
:102440000028E6D0F4E71FBD2442020010B5044C7A
:102450002078002803D001F0B3F80120607010BD8F
:10246000B8280020016009684160AFF3008010B512
:10247000D0E900215368994201D1002104E0D1E95B
:102480000034A34202D01946816010BD083141607A
:10249000F0E7816800290BD0026892680A448260E4
:1024A00041684B689A4203D108314160FFF7DFBFB2
:1024B00070474058002800D00120704708B500221E
:1024C00042504058009008BD08480068012110F0B3
:1024D000010F08D14FF0E020E02280F80024C0F87E
:1024E0008012C0F8001102480160704700E100E06E
:1024F0001805004010B54FF48070FFF7E4FC012090
:102500008107C1F80403086010BD000006490246B7
:1025100000200B790BB1852070470A6001220A71F7
:1025200000224A71704700009C27002004490120C6
:10253000086004480168C1F300410029FAD17047DE
:102540000C00004018040040002802D0014980011E
:1025500008477047093F02000121B1EB507F01D1CC
:10256000012070470020704700207047704700002E
:102570002DE9F0410546164600790F46154A00EB55
:10258000C00102EB810494F8201011B10820BDE8CD
:10259000F081114951F820102868FFF7E5FF08B1D4
:1025A0001120F4E739462846F7F74AFA6660386999
:1025B00020601EB1397F2846FFF72CFB28680821D0
:1025C000C0F800150020A061E0610121606184F87D
:1025D0002010DCE7EC330020043F02002DE9F05F1F
:1025E000044600790E4600EBC001DFF8F0A0174664
:1025F0000AEB81053046FFF7AFFFB0B168684FF0D6
:1026000000084FF4047910B12168C1F80893A86953
:102610004FF0000B80B1E86948B1686810B12068DC
:10262000C0F804931120BDE8F09F1020FBE7EF6194
:102630004FF001082E6102E0EE60C5E9067B00253F
:102640004FF488712068FFF739FF4FF4A2712068BA
:10265000FFF734FF2068C0F83465C0F8387520688B
:10266000B8F1000F12D0D0F8001241F02001C0F8EC
:1026700000122079D04600EBC0010AEB81004068CF
:1026800038B12068C0F804932846CCE701210160E6
:10269000EFE74FF4887A4FF4A27951462068FFF7AC
:1026A00008FF074649462068FFF703FF06464FF438
:1026B00092712068FFF7FDFE014647EA06000843D5
:1026C000EBD0227902EBC20308EB8302C2F818B008
:1026D00001B10325002ED7D00F25D5E7EC3300201C
:1026E0002DE9F04704460E460079204900EBC00072
:1026F00001EB800517463046FFF72EFF30B120462C
:1027000000F036F820B11120BDE8F0871020FBE77B
:102710006F61AE604FF49076002731462068FFF776
:10272000CDFE4FF4AC7841462068FFF7C7FE206825
:10273000AA686969C0F84425C0F8481520680121D5
:102740008160686878B9B14649462068FFF7B1FEF4
:10275000064641462068FFF7ACFE0643F4D000B1C0
:102760000F27002068613846CEE70000EC330020D8
:102770000079054900EBC00001EB800040690028AA
:1027800000D0012070470000EC3300202DE9F04715
:1027900004460079274900EBC00001EB8007206860
:1027A0004FF00009C0F80095786880B12068224990
:1027B000C0F8081320680121000B40B200F01F028E
:1027C00091404009800000F1E020C0F880112068AD
:1027D000D0F80C25D0F81485D0F80865D0F810553D
:1027E0004FF0FF31C0F80C15C0F814152068C0F880
:1027F0000815C0F81015501C02D01046FFF749FC10
:10280000B8F1FF3F02D04046FFF743FC681C02D0FE
:102810002846FFF73EFC701C02D03046FFF739FC1B
:102820002068FFF7A3FE87F82090C7F80490BDE862
:10283000F0870000EC3300201003020041DF002885
:1028400001D0F6F7E1BF704770B51D46049C0E46F7
:10285000034642B13DB134B129682068091A0529FF
:1028600003D2092070BD0E2070BD411C216013549D
:1028700020688118304601F03BFA21680844206046
:102880002860002070BD00002DE9F05F5E4D00263D
:102890000B464FF0050B3446C0B2297804276BF382
:1028A00007044FF003084FF002094FF0010A072810
:1028B00063D2DFE800F00413535E7A8289006878FF
:1028C00003285AD16F70514800F014FC08B1F6F794
:1028D0009BFF3146204661F3070048E020469AB24C
:1028E0006AF30700B2F5007F19D8012902D0042944
:1028F0000ED042E032466B6811469847444800F0DB
:1029000001FE08B1F6F780FF85F80090BDE8F09F62
:1029100032466B681146984785F800B0F6E7012902
:1029200002D004290DD028E032466B681146984742
:10293000002000F0E7FD08B1F6F766FF85F800809B
:10294000E4E732466B6811469847002000F0DAFD54
:1029500008B1F6F759FF06202870D7E702290CD1F5
:1029600020462F7069F30700194662F30F063246BE
:1029700045E0032906D006290ED0BDE8F05F00200F
:10298000F6F742BF204632466B6868F307001146EF
:10299000984785F800A0B9E7204632466B6868F38F
:1029A0000700114698472F70B0E73246204611467F
:1029B00067F3070062F3070121E02046314667F321
:1029C00007006AF30701D2E767F307046878A046B7
:1029D00069F307061C46032802D0022905D00BE044
:1029E0006F70104600F086FB03E02F70104600F079
:1029F00037FB08B1F6F708FF2246314640466B68C0
:102A0000BDE8F05F184700004C280020084900206E
:102A1000084B002028B111B10078332803D00720DB
:102A200070470E207047012901D00920704700200F
:102A3000704701680A684968914201D3881A704753
:102A40008068801A0844401C7047000070B52A4C0A
:102A5000617A6069FEF724FC012510B1E58104204C
:102A600070BD00F07DF82549606908602348617AEF
:102A7000001D016021481830026822F0FF02026048
:102A80000368A26A43EA1263036010021B4A103211
:102A900010601A4824300560184A00202032106067
:102AA000207AA27940EA0220144A283210600329D1
:102AB00001D004290CD12079E178000440EA0120FA
:102AC000A1780843617940EA01600C490831086047
:102AD00094F8240094F82010400640EA0160A18B8D
:102AE00040EA0140E17940EA0120044940F0FF005A
:102AF0000C310860002070BD502700200C150040EC
:102B000010B50446FEF770FC1149124AC86A1060FD
:102B1000121D086B1060086C022202EB40000D4A87
:102B2000303A1060121F0C4810600C4A0020C2F8A6
:102B300000010323C2F8003224B1C2F80C010120C5
:102B4000506010BD486903492C39086010BD000071
:102B50005027002038150040D432002000100040DB
:102B60000B49032008600B490020C1F80002C1F89E
:102B700010010122C1F81020D1F81021002AFBD049
:102B8000C1F810014860086003498881704700005F
:102B900008F50140001000405027002070B50126C4
:102BA00070044FF0E0210025C1F88001084C40106E
:102BB000C4F84803C4F8080366602F20FFF7C4FC7C
:102BC000A660044C2F20A560FFF7BEFCA57070BD69
:102BD00000100140B827002010B5017842788378B2
:102BE000C0780A441844104410F0FF0F0ED1C1F30E
:102BF000C204FEF7BFFCA04206D0FEF7BBFC401C9F
:102C000000F00700A04201D1012010BD002010BD3E
:102C10001FB501238DF800308DF808100192D0E91E
:102C20000012684690471FBD70B50D460446F6F782
:102C300089FD70B12846F6F797FD68B16807000E68
:102C4000002C0CDA04F00F0101F1E02181F8140DE1
:102C500009E042F2010070BD42F2020070BD04F1D1
:102C6000E02484F80004002070BD000038B5002185
:102C7000012548B101280CD0032809D1FFF724FC15
:102C8000BDE83840FFF788B94FF0E020C0F8805128
:102C900038BD8DF800106846F6F794FE064C207893
:102CA00008B9FFF75DF9E068401CE060A5709DF889
:102CB0000000F6F7ABFE38BDD83300203EB5044621
:102CC00009496846FFF7CEFB08E000BFD0E90021C4
:102CD0002046904730B16846FFF7DBFB029800289A
:102CE000F4D13EBD11203EBDA04102003EB50446D8
:102CF00008496846FFF7B6FB07E000BFD0E90021AE
:102D0000204690476846FFF7C4FB02980028F5D19B
:102D10003EBD0000AC41020010B51C460B462AB176
:102D200024B12168052903D2092010BD0E2010BD51
:102D30001070511C184600F0DBFF401C2060002082
:102D400010BD00001CB5040002D10E20F6F75CFD9A
:102D5000002001900090694601A800F0ADF9042818
:102D600020D008B1F6F750FD019A02206B4602F818
:102D7000010B00980021401E00902046F7F731F823
:102D8000062812D008B1F6F73FFD0098401C81B22A
:102D90000090019800F0C8F908B1F6F735FDF6F794
:102DA000D7FD1CBD00F0DAF8D5E7019800F0A2F9D4
:102DB00008B1F6F729FD0248F6F726FD1CBD000014
:102DC000FECADDBA10B54188074AF6F729FD08B1F9
:102DD000F6F71AFDF6F7D0FD002803D1BDE8104044
:102DE000FFF734BB10BD0000452D02007FB50E4635
:102DF00004000DD07EB10020029001902578039050
:102E000001A902A800F058F9042806D040B122E038
:102E10000E2004B070BD0920FBE700F09FF8EFE73B
:102E2000029A012001AB02F8010B01983146401EC5
:102E300001902046FEF72AF806280BD10C48F6F739
:102E4000E3FC03A8029A009001AB06212846521C1D
:102E5000FFF7FAFC08B10320DBE70198401C81B2C0
:102E60000190029800F060F90028F4D1D1E7000049
:102E7000FECADDBA7CB50D46040017D000200190D3
:102E80000090694601A800F017F9042810D0002826
:102E90000DD101990420134A087000982946401E5C
:102EA00000902046F6F74EFF28B118E00E207CBDBA
:102EB00000F054F8E5E701996A460020491CF6F74E
:102EC00067FF60B90098074A401C521E012100901C
:102ED000117081B2019800F027F90028E7D0032093
:102EE0007CBD00003528002010B5C0B2052813D2E3
:102EF000DFE800F003090D131500F6F74FFDBDE8FC
:102F0000104000F015B8BDE81040F6F721BD0648A6
:102F1000C0E902120121017010BD044800E00F2039
:102F2000BDE81040F6F770BC3C280020FECADDBAB0
:102F30001CB5094C207800280DD011DF00F062F894
:102F400054F8010F0090A188ADF804100199BDE874
:102F50001C40FEF7E1B91CBD34280020024840683F
:102F6000002800D0004770473C28002001494860F5
:102F7000704700003C28002010B504001ED02268D5
:102F8000A188501C491E127889B23AB1032A08D090
:102F9000052A0AD00A48F6F737FC08E0FFF726FFB3
:102FA00001E0FFF767FF10B106E000F00BF82068C2
:102FB00000F056F8002800D0032010BD0E2010BDF0
:102FC000FECADDBABFF34F8F05480168054A01F418
:102FD000E06111430160BFF34F8F00BFFDE70000C8
:102FE0000CED00E00400FA05054900200A78002AEB
:102FF00004D0087001F10800FFF7BEBF7047000061
:103000003C28002010B500F0EFF9044800210170C1
:1030100041704160BDE8104000F02AB94C28002002
:1030200010B50D4C21786278114301D0082010BDF5
:1030300080B10121217061706060084800F038FAA9
:103040000028F4D000212170617061600728EED063
:10305000032010BD0E2010BD4C280020892802003E
:1030600070B50546002400F0BFF925B1104885422F
:1030700003D010240AE00E2408E00E4D287804281E
:1030800008D0062808D0052808D0082400F0BEF98A
:10309000204670BD012009E0032007E0044800F04D
:1030A00031FA040001D00324F0E702202870EDE794
:1030B000084B00204C28002010B502004FF0000003
:1030C00007D031B1094C63782BB1012B05D0042016
:1030D00010BD0E2010BD082010BD02236370044BEC
:1030E00013604FF400720A8010BD00004C280020CD
:1030F0000849002001004FF0000004D0084A914226
:1031000003D0102070470E20704706494A78022AE3
:1031100003D0042A01D00820704701224A7070476A
:10312000084900204C28002070B50C46050005D049
:1031300034B11348854205D010240DE00E240BE075
:10314000072409E0B4F5007F01D90C2404E00D4EFA
:103150007078022802D00824204670BD00F044F99F
:103160002146284600F0E6F9040005D0112C00D0D5
:10317000032400F04BF9EFE703207070F9E700003B
:10318000084900204C2800202DE9F843364C8DF8E2
:1031900000004FF0010C6178002511B1216A39B1AE
:1031A00008E0C02802D1256284F801C0BDE8F88398
:1031B000C028FBD02C4ADFF8B490E768126940F2CF
:1031C0000623022627B194F80280B8F1000F08D038
:1031D0007AB384F802C06261994230D3C02840D1EA
:1031E0002DE031B1042906D099420DD3C02838D141
:1031F0000AE0676108E0C02806D0D2B11B48E16A46
:103200003038816778306061684600F0ADF950B1C0
:10321000A07A0028CAD16269206A9DF80010115472
:10322000401C2062C2E76169E068814202D1E5602A
:1032300001E016E02561484689F800600AE068462A
:1032400000F092F90028E3D12561A57089F80060AB
:10325000616948464160218CA9F80810616A0348F9
:1032600088476570A2E7000088280020704F002082
:1032700070B5044C0025A56100F00EF8257065704E
:1032800070BD000054280020024B9B69002B00D029
:10329000184770475428002010B50348FFF776FA06
:1032A00002490020486210BD6441020088280020C5
:1032B00010B520B1154C616A19B1082010BD0E205F
:1032C00010BD14496062124AA1F10C00FEF77CFEA9
:1032D00008B1072010BD1048A0620020E07007214F
:1032E00021716071A071A072084808492C30E0601B
:1032F000094801223C302061064809310C38FEF7AC
:1033000083FE08B1F6F780FA002010BD882800205F
:10331000413A02006C4102007C4F002001004FF056
:10332000000007D00A4BA3F12C02994208D1D168C2
:1033300011B103E00E207047D3607047082070473A
:10334000044B9942FBD111690029F7D113617047F1
:10335000B4280020B84F0020F8B515460E460700E7
:103360001BD000248DF800406846F6F72BFB1C4963
:103370000A791C48072A16D0D7E90012C0E90612BC
:1033800000F118015EB1D6E90023C0E9082345B178
:10339000D5E90012C0E90A1217E00E20F8BD8C60D2
:1033A000F5E70C6111E0D7E90023C0E900230D4ADD
:1033B0008EB1D6E90036C0E9023675B1D5E90023F1
:1033C000C0E904230C7100F08DFA9DF80000F6F7B7
:1033D0001DFB0020F8BD9460EFE71461F2E70000E8
:1033E00088280020404F002038B500248DF8004088
:1033F0006846F6F7E7FA04484471C4719DF8000086
:10340000F6F704FB38BD000054280020F8B500266C
:1034100035468DF800606846F6F7D4FA224C01274D
:103420006771A07908B1A57101269DF80000F6F733
:10343000EDFAE7718DF800506846F6F7C3FA1B48BD
:10344000FEF713FFA178E279114208D038B1A570D8
:103450009DF80000F6F7DAFAFEF734FB03E09DF87A
:103460000000F6F7D3FA8DF800506846F6F7AAFA8E
:103470000E481430FEF7F9FEE178E279114208D0E7
:1034800038B1E5709DF80000F6F7C0FAFEF782F952
:1034900003E09DF80000F6F7B9FA002E03D0BDE86E
:1034A000F840FEF71FBAF8BD542800205042020031
:1034B00070B5114C054620786178084301D008208A
:1034C00070BD25B1FEF7B0FA18B1032070BD0E2013
:1034D00070BD0A48FEF7B8FE08481430FEF7B4FE87
:1034E0000748FFF7E5FE0028F2D16062A5610121DF
:1034F000A0622170617070BD54280020504202000B
:10350000FD1802001FB50A4900240A795AB10022A9
:103510000A71086101208DF804008DF800206846CA
:10352000FEF710F900E0112404B0204610BD0000A1
:10353000542800201FB5002438B131B1094A53691D
:103540002BB11124204604B010BD0E20FBE7918161
:10355000506100208DF800008DF804006846FEF7E9
:1035600089FAEFE75428002010B50478C02C0AD05F
:103570000C49DB2C09D00A460023927ADC2C07D0B8
:10358000DD2C0DD108E0002010BD0120887207E07D
:1035900032B18B72C02102E012B18B72DB2101705B
:1035A000012010BD88280020002805D103490120F2
:1035B00048700020FCF72ABA70470000D83300207A
:1035C00010B51620F6F7BEF848B10A4882684FF4E5
:1035D000800152B1016821F48001016010BDBDE895
:1035E000104042F20100F6F70FB94FF0E020C0F8AA
:1035F000801110BD1C35002010B51620F6F7A2F87A
:1036000080B10F4890F800044009F6F7ADF860B1BA
:103610000C4882684FF480016AB1016841F480016E
:10362000016010BD42F2010001E042F20200BDE87B
:103630001040F6F7E9B84FF0E020C0F8001110BDD7
:1036400016E000E01C3500207CB50C4640B12CB1E2
:1036500000230193057801A94C2D03D007207CBDE0
:103660000E207CBD0125CDE9003513460A462146D2
:10367000FCF744FA0028F4D10198A04201D00920B7
:103680007CBD00207CBD00002DE9FF4184B0984640
:1036900014460F0019D0C4B10020019025684C20B9
:1036A00001AE8DF8080033462A4602A800F06EFBF2
:1036B00000280BD133462A46394604A800F038FBCF
:1036C000002803D1049870B903E00E2008B0BDE8CB
:1036D000F0810748009033462A4639464046FCF7B9
:1036E0003BFA0028F2D1019820600020EEE70000AC
:1036F000313D020010B54FF080400021C0F80011AC
:1037000001220260D0F80031002BFBD0104B9869E9
:103710004260C260C0F80415C0F84011C0F84411FE
:10372000C0F84811C0F84C114FF48034C0F804437D
:10373000C0F800220424C0F810455C6BC0F8404576
:103740004FF48274C0F8444502600020196110BD36
:10375000502700202DE9F84F1D4C00256846D4E97C
:1037600001A6FDF7E7FE002738B30023009A616841
:103770001CE0D1F800C00846944503D9ACEB020226
:103780000A6015E0A2EB0C0263440760D0F80CC09D
:10379000C1698146BCF1000F08D006EB030828F090
:1037A0007F48C0E9018CC9F81C5005460029E0D1CA
:1037B00028466160FEF7C2FA03E02846FEF7BEFA2B
:1037C00010B15046FCF744F9E770BDE8F88F0000EF
:1037D000B82700200D4B10B5596831B102680C684C
:1037E000A24204D8A21A0A60C161586010BD0B46FB
:1037F00003E00B46C969121B21B10C689442F8D34F
:10380000A41A0C600260C161D86110BDB827002005
:103810002DE9F041144E77683D462C4603E0844282
:1038200004D02546E469002CF9D11BE0D4B1A542AF
:103830000BD1F869706040B90C4901208860002103
:10384000B160F0702F20FEF77FFE2168E069E8612B
:1038500010B10268114401607068874202D00120F3
:10386000BDE8F0810020FBE7B827002000100140F0
:103870002DE9F041194D6C68002C2CD01848002718
:103880000068A968B846401A20F07F462068B04218
:103890000CD82146361A0744E469087C20B181F827
:1038A0001080886949698847002CEFD129786878A9
:1038B000814206D1401CC0B26870022801D185F84F
:1038C0000180064869780C3040F82170BDE8F0416D
:1038D0001420F5F741BDBDE8F0810000B8270020B5
:1038E000041501402DE9F047DFF8DC900126374C44
:1038F000A9F1180700254FF00508207818B100F04D
:1039000067F806461AE0207980B1042818D0052807
:1039100016D006281AD0A069E1690068405C491CED
:10392000E161C02824D0DB2825D026E0C02000F0AB
:103930004FF8C4E90675064601202071257034E071
:10394000C02000F045F8064684F80480D9F800004D
:1039500048B11D491822A1F11800F5F76DFCC9F80E
:103960000050257121E02079401C2071BDE8F087CE
:10397000DB20DC2100E0DD21217000F029F8064683
:10398000A069E269818891420FD8056020790128F9
:1039900003D0207902280DD014E0B86840B10A485D
:1039A0001038C4E9060502202071002EA5D1DDE7FC
:1039B0000420F9E7386928B103480838C4E9060546
:1039C0000320F1E74046EFE7584F00208828002009
:1039D00070B5184CE278A16A8854521CD2B2E270D9
:1039E00023790420042B0BD02379052B0AD01E2A1F
:1039F0001DD3657901233DB12072A371002070BDF4
:103A00000120F6E70020F4E76371E0710A48FEF751
:103A100001FB08B1F5F7F8FE0849A06A884202D117
:103A200001F11E0000E00548A0620020E0700120C6
:103A300070BD000088280020604102007C4F0020FB
:103A400070B501782D4D2E4CD1B1012945D00229F8
:103A500001D0032010E0C068810705D00321297040
:103A60006860616A2548884725490122093125484F
:103A7000FEF7CAFA002840D0BDE87040F5F7C4BE92
:103A8000A0790026C8B1E2781E48A16AFEF7C2FA02
:103A900008B1F5F7B9FE1949A06A0C31884202D184
:103AA00001F11E0001E015480C30A062E670E079DB
:103AB0002870207AE071A67102E06671E0792870C2
:103AC0002878042802D0616A0C48884720790728A2
:103AD00013D0BDE87040FFF705BF09480122093047
:103AE000014604780748FEF78FFA08B1F5F78CFE17
:103AF0002046BDE87040FFF747BB70BD704F002007
:103B0000882800206041020010B50446407988B042
:103B10000A2802D9072008B010BD202213496846A0
:103B2000F5F78AFB20780190607800906079104961
:103B300051F82000069000208DF814008DF8150033
:103B400001F15C00FEF722FE094800226946583068
:103B5000FEF73AFA0028DED1054960792C3151F898
:103B60002000303908600020D5E700004041020005
:103B7000D02700201FB50A4601788DF80010416853
:103B80000191017A8DF80810C0680390044850F83C
:103B90002210001F50F82220684690471FBD0000E9
:103BA000982700202DE9FF410C464FF492770546F7
:103BB0003946FEF77EFC0026C0B139462846FEF79E
:103BC0007DFC02208DF80000D5F88004C5F8800443
:103BD0000390D5F83C058DF80800E0680190A661D7
:103BE000E661D4E900126846904723E04FF48877F5
:103BF00039462846FEF75DFCE0B139462846FEF717
:103C00005DFCD5F83C15A069884213D1E06960B12C
:103C1000E268D5F8000220F02000C5F80002E06953
:103C2000A0612069E661E06001E0A661E2682046EB
:103C3000FEF7EEFF4FF4A27739462846FEF739FC2F
:103C400060B139462846FEF739FCA06930B1A6615B
:103C5000D5F83C152046E268FEF7DAFF4FF490777E
:103C600039462846FEF725FC002813D03946284659
:103C7000FEF724FC606900280CD0D5F84C058DF8BF
:103C800000608DF80800A06801906661D4E9001218
:103C900068469047BDE8FF8130B51468A51C8D4289
:103CA00005D82044008818801068801C106030BD42
:103CB00010B51468091B022901D2092010BD204447
:103CC000008818801068801C1060002010BD10B59E
:103CD0001C68121B022A01D2092010BD2144008851
:103CE0000870000A48701868801C1860002010BD19
:103CF0000870020A4A70020C8A70000EC870042014
:103D0000704710B538B132B12BB11468091B0429C2
:103D100003D2092010BD0E2010BD2044C1780068D8
:103D200061F31F6018601068001D1060002010BD56
:103D300010B51C4639B130B12CB12368D21A042A0F
:103D400003D2092010BD0E2010BD19440068FFF7F2
:103D5000CFFF216808442060002010BD30B51468F2
:103D6000651C8D4204D8005D18701068401C1060FE
:103D700030BD10B514688C4201D1092010BD005D22
:103D800018701068401C1060002010BD10B51C6831
:103D9000944201D1092010BD007808551868401CD4
:103DA0001860002010BD70B51446049D2BB1226828
:103DB000891AA94203D2092070BD0E2070BD1118C6
:103DC0002A461846F5F738FA206828442060002073
:103DD00070BD70B50D46049C38B132B12CB121686C
:103DE0005B1AAB4203D2092070BD0E2070BD8B1848
:103DF00001462A461846F5F71FFA20682844206035
:103E0000002070BDFFC1FBE84C90728BE7B3518975
:103E100063AB232302841872AA612F3B51A8E537B4
:103E200049FBC9CA0C18532CFD45E39AE6F15DB075
:103E3000B61BB4BE2A50EAE90E9C4B5E5724CCA1B7
:103E4000B759B887FFE07D742648B9C5F3D9A8C42F
:103E5000B1D5911101420C39D5B0979D28D4F29B70
:103E6000A4FD6465068C2996FEA2714DF3F82E58C8
:103E7000DB0D5A5F1528F57407CE25AF2B12E6D05F
:103E8000DB2CDCC37FF03E3A13A4DCE2F96C54E295
:103E9000D8EAC8880021869C6AD8CB4E146AF94DAE
:103EA000D27EB23203C6144B7FD1B8A6797C17AC50
:103EB000ED06ADAF0A947ABA03E792D7150973E815
:103EC0006D16EEE13F781F9D09526EF17C362A7126
:103ED0006C7564448010434E35EC65270AB5FC26AA
:103EE000693F599901638AA5BF685CD33CBE0BD674
:103EF0007683D657054A3DDD8173C9EB8A8439F450
:103F0000360BF700159701000738FDD87047000001
:103F100033000000C90E02004C000000E30E020056
:103F2000460000005B0E020062000000EF0D020080
:103F300063000000510D020064000000990D0200B2
:103F4000650000002B0E0200680000002D0C02002E
:103F5000670000007D0C02006000000099FD010078
:103F600066000000E50C0200690000004DFD010044
:103F70006C000000FDFD01006D000000CDFD0100A2
:103F800070000000E302020071000000AB020200BA
:103F90006E000000090502006F0000001900020019
:103FA00086000000C30302007300000085FE0100CC
:103FB00074000000B5FE010075000000AFFF0100B5
:103FC000760000000501020077000000CD04020029
:103FD0007800000011FF010079000000E1FE0100FF
:103FE0007A0000007F0202007B0000004F02020006
:103FF0007C000000BF0002007D0000008300020082
:104000007E0000007BFF01007F0000001104020021
:10401000800000003BFF010086000000C303020097
:1040200087000000E3FF0100880000005F0302003A
:10403000890000009903020082000000350102009F
:10404000810000006501020084000000DD01020023
:10405000830000009B0102008E0000001703020095
:104060008F0000001D0202007200000029FE010006
:104070009B000000E90602009C00000065070200AA
:104080009D0000001F0602009E0000005306020073
:10409000A000000093050200A10000002907020013
:1040A000A2000000D9050200A30000009907020049
:1040B000A4000000B90602009F0000005B0502009A
:1040C000A500000087060200A8000000650A0200A3
:1040D000A9000000AF090200AA00000027080200A2
:1040E000AB000000CB080200AC000000D90B0200BE
:1040F000AD0000008D0B0200AE0000005709020069
:10410000AF000000AB0A0200B00000001F0A02006E
:10411000B10000003D0B0200B2000000E50A020001
:10412000B3000000F1090200B4000000E107020042
:10413000B500000025090200000200000000000098
:10414000FFFFFFFFFFFFFFFFFFFFFFFFFFFFFFFF7F
:1041500000000000000000000000D6010700000081
:1041600000000000002000400000000017000000D8
:10417000180000001900000002000000000000000C
:10418000010E000000000010070000000000000009
:104190000000000000000000000000000100000717
:1041A0008C4102009C41020008000000C441020052
:1041B000D441020008000000D4410200E4410200A2
:1041C0000800000098420200A04202000000000027
:1041D0000000000088420200984202000000000037
:1041E000000000007842020080420200000000004F
:1041F00000000000000000000000000000000000BF
:104200000000000050270020E441020004420200A8
:104210000800000080420200884202000000000006
:1042200000000000144202002442020008000000C6
:10423000A04202005027002070010000C09201003F
:1042400004430200C0280020003100003497010020
:10425000184E0020084D0020100000001000000043
:1042600001000000344F0020244E00201000000008
:104270001000000001000000C52D02000000000039
:10428000A935020000000000A52202000000000085
:1042900011240200000000006D2C0200000000004C
:1042A00011240808011201F303031280AA40132706
:1042B000294176715B06145555550346C4094233AE
:1042C00023F0041AD05123B0131B502710223A2395
:1042D000A04E33C075329D22EB1B903AA42BD60121
:1042E000303223321B32175A15045A1404194279FA
:1042F000045112200226401301012902016004002A
:0443000090D0030056
:040000050001920163
:00000001FF
